:10678B000000090200000301FA0400FA0500030AE5
:10679B000A5A0B001E0C00FA0D00030E00040F0129
:1067AB0064100096120132130AFA14010217010A3F
:1067BB001801FA1905321A010A1B01FA1C05321FBE
:1067CB00FFFF20FFFF23011E2400642A00FA2B0089
:1067DB00FA2C50782D003D2E004630006432507854
:1067EB003300003432FA3501643601643701503816
:1067FB000A643C00643E003C3F000140FFFF411433
:10680B0050420A5A430AC84405324500B44600FABE
:10681B004C00FA500404510596520A32530B46545D
:10682B000A96570546590A465A32FA5B010A5C0A20
:10683B00325E000A5F00FE64021067FFFF6A0A3CCB
:10684B006B00006C32967300017400017801327991
:10685B0001327E006481006484FFFF8A00019D0A7F
:10686B00969E00019FFFFFA00124A2000AA3FFFF39
:10687B00A4FFFFA5FFFFA6FFFFA7FFFFA8FFFFA930
:10688B00FFFF0101481500022F003C470148480259
:10689B00035601044EFFFF58000261FFFF66000222
:1068AB008500AF8600018700FA89010A990008A1CB
:1068BB0000FAFAFAFA0101241500022F1E3C4701D7
:1068CB00484802035601034EFFFF58000261FFFFC9
:1068DB006600028500AF8600018700FA89010A99DC
:1068EB000000A10000FAFAFA0065006F007900833E
:1068FB00008D009700A100AC00B600C000CA00D408
:10690B0000DE00E800F200580060006800700078BC
:10691B00008000880090009800A000A800B000B88C
:10692B0000C100C800D000D800DF00E600EE00F682
:10693B0000410047004D00530059005F0065006C9B
:10694B0000710077007D00830089008F0095009B0C
:10695B0000A200A700AC00B200B900C000C500CA7D
:0C696B0000D200D500DD00E100E700EFE5
:10331000900885E0900111F0900886E0900080F020
:10332000900887E09000A0F0900888E09000C9F035
:10333000900889E0900075F090088AE09000BBF05A
:1033400090088BE09000D9F090088CE09000ADF0F0
:1033500090088DE09000CBF090088EE09000FBF09C
:1033600090088FE090015FF0900890E0900160F08D
:10337000900891E0900161F090015FE0700C900185
:1033800060E07006900161E060028004C22080026B
:10339000D220745390014AF0747590014BF074621E
:1033A00090014CF0746190014DF0747290014EF0F8
:1033B000747590014FF07420900150F074349001B6
:1033C00051F07443900152F07479900153F0746C91
:1033D000900154F07420900155F07433900156F030
:1033E0007436900157F07454900158F02290087D83
:1033F000E0FEA3E0FF7402D39F74019E400C90672F
:103400008B120048E493F599802F90004BE0D39401
:1034100005401490087DE0FEA3E0FF90678B12004A
:1034200048E493F599801290087DE0FEA3E0FF90B8
:1034300067BE120048E493F59990087D126A979050
:10344000087DE0FEA3E0FFEFB43507EEB40103759D
:103450004D002285F97385FA747E017F00E57412B0
:103460006A89E5732FFF50010E8E5A8F5B9000150D
:10347000E0FCA3E0FDEF2DFDEE3CFC8C5C8D5D22BD
:1034800075A71085F97385FA747E017F00E57412C3
:103490006A89E5732FFF50010E8E5A8F5B9000D919
:1034A000E0B40210AC2CAD2DEF2DFDEE3CFC8C5C9D
:1034B0008D5D8016AE5AAF5B900015E0FCA3E0FD79
:1034C000EF2DFDEE3CFC8C5C8D5D22AE5AAF5B7443
:1034D0000A8E048F05FF126A798C5C8D5DAE5AAF3F
:1034E0005B740A8E048F05FF126AA48C5A8D5BC22E
:1034F00000E55B455A6013740AC3955BFFE4955A77
:10350000FE8E5A8F5B785C126ADCE573A85CB800AB
:1035100015D3955D4010E573C3955DFFE4955CFEA2
:103520008E5C8F5D8012E5732424C3955DFFE49566
:103530005CFE8E5C8F5DD200757300AE5CAF5D7417
:10354000116F4E600674126F4E7018AE5CAF5D74F2
:10355000116F4E70057573018003757302755D10F0
:10356000755C00AE5CAF5D74146F4E600674156FD1
:103570004E7018AE5CAF5D74146F4E7005757301BC
:103580008003757302755D13755C00AE5CAF5D748E
:10359000236F4E600674246F4E7018AE5CAF5D747E
:1035A000236F4E70057573018003757302755D227C
:1035B000755C0022900087E0B40104C2078002D24B
:1035C00007900088E0B40104C2088002D20890008D
:1035D000C5E075F0E1A4FFAEF0740A8E048F05FF1C
:1035E000126A79900875ECF0A3EDF074078C068DE3
:1035F00007126A8974038E048F05FF126A7990009E
:1036000011ECF0A3EDF07E017F00900083E0126AE0
:10361000899000C6E08E048F05FF126A79740AFF54
:10362000126A798D609000CFE075F0E1A4FFAEF0F2
:10363000740A8E048F05FF126A79900879ECF0A362
:10364000EDF09000D1E060139000D1E0F5F0741639
:1036500084FF7E00EF9008A1F0800674649008A1BA
:10366000F09000C7E0900062F0900113E090006DD0
:10367000F0900115E0FE9000C3E08E0088F0A4FFFA
:10368000AEF0EF9008A9F0900111E0900885F0905D
:1036900000A0E0900887F0900075E0900889F09015
:1036A00000FBE090088EF090015FE090088FF090B2
:1036B0000160E0900890F0900161E0900891F0A224
:1036C00020B3401690015FE0700C900160E070063E
:1036D000900161E060028002C22090015FE0B4309E
:1036E0000F900160E0B44708900161E0643B600224
:1036F0008004D2218002C22174E3900061F0900026
:10370000B0E0B40B0874E3900061F0805A9000B010
:10371000E0B419129000C6E09068DE12008CE493C9
:10372000900061F080419000B0E0B41E129000C69D
:10373000E09068FC12008CE493900061F080289087
:1037400000B0E0B428129000C6E090692612008C08
:10375000E493900061F0800F9000B0E0B4460890D0
:1037600000A7E0900061F0900088E070089000C928
:10377000E064046002800874039000C9F0D21F90D6
:103780000065E0FE9000ADE0B50657900067E0FEF2
:103790009000CBE0B5064B900066E0FE9000D9E0CB
:1037A000B5063F90006AE0FE900080E0B5063390D9
:1037B0000068E0FE9000BBE0B50627900069E0FEDF
:1037C0009000C9E0B5061B90006BE0FE9000E6E0BB
:1037D000B5060F90006CE0FE9000E7E06E7003020B
:1037E00039C590004BE0C39405500874029000FC6A
:1037F000F080149000D9E0600874069000FCF0801E
:1038000006740A9000FCF0900080E0B40106740099
:10381000900080F0900080E0B4020674009000CB2D
:10382000F0900080E0B4030674009000D8F090009F
:10383000CBE0D394014027741B9000FEF0740090FD
:1038400006C9F074009006CAF07400900095F090DC
:1038500000ADE0B4020674019000ADF0803390003A
:10386000ADE0B4021A74009000FEF074009006C936
:10387000F074009006CAF0741B900095F0801274EA
:10388000009000FEF0741B9006C9F0740090009543
:10389000F09000ADE06014741C900094F0740090FF
:1038A00006CDF074009006CEF0800C740090009469
:1038B000F0741C9006CDF09000E6E060147419904E
:1038C0000100F074009006C1F074009006C2F08010
:1038D0000C7400900100F074199006C1F09000E79C
:1038E000E06014741A900101F074009006C5F07441
:1038F000009006C6F0800C7400900101F0741A90DC
:1039000006C5F09000D9E0701A74059006D1F074E5
:10391000069006D5F074079006D9F074089006DD7D
:10392000F0803074009006D1F074009006D2F074EC
:10393000009006D5F074009006D6F074009006D979
:10394000F074009006DAF074009006DDF0740090D8
:1039500006DEF0D21F9000ADE0900065F09000D937
:10396000E0900066F09000CBE0900067F09000BB24
:10397000E0900068F09000C9E0900069F09000804D
:10398000E090006AF09000E6E090006BF09000E7B5
:10399000E090006CF0900080E0900886F09000C904
:1039A000E0900888F09000BBE090088AF09000D981
:1039B000E090088BF09000ADE090088CF09000CB88
:1039C000E090088DF09000E3E0B4011790002174BE
:1039D0000FF0A374FFF0900023E4F0A3F0740290C2
:1039E00000E3F09000E3E0B40341900023E0FEA385
:1039F000E0FF900021E0FCA3E0FD126AD4741012F5
:103A00006A897408120039EF90005EF0EF70067456
:103A1000FF90005EF074009000E3F0900022E090D0
:103A2000005FF0900021E0900060F0900074E09062
:103A30000071F0900073E0900070F09000A2E0C37D
:103A4000941E50569000A2E0F404241E900072F0E0
:103A5000900072E075F00A84FF7E008F7390007210
:103A6000E075F00A84ADF07C008D74900070E0D3B6
:103A70009574400D900070E0C39574900070F080D4
:103A80000F900070E0240AC39574900070F00573E5
:103A9000900071E02573900071F0900071E090004B
:103AA0003DF090003DE0241290003EF090003DE09B
:103AB000D39448400B90003DE0C3944890003DF003
:103AC00090003EE0D39448400B90003EE0C3944801
:103AD00090003EF0C22390003DE0D39424400D902E
:103AE000003DE0C3942490003DF0D223C224900016
:103AF0003EE0D39424400D90003EE0C39424900017
:103B00003EF0D224900041E4F090003DE06411606A
:103B10000790003DE0B4122090003DE0B41106741F
:103B200002900041F090003DE0B412069000417414
:103B300001F0741390003DF090003DE064146007C4
:103B400090003DE0B4152090003DE0B414067402EE
:103B5000900041F090003DE0B415069000417401E2
:103B6000F0741690003DF090003DE06423600790F3
:103B7000003DE0B4242090003DE0B42306740290A0
:103B80000041F090003DE0B424069000417401F043
:103B900090003D7401F0900042E4F090003EE0643B
:103BA00011600790003EE0B4122090003EE0B41196
:103BB000067402900042F090003EE0B412069000BD
:103BC000427401F0741390003EF090003EE06414E3
:103BD000600790003EE0B4152090003EE0B414066B
:103BE0007402900042F090003EE0B415069000424E
:103BF0007401F0741690003EF090003EE064236083
:103C00000790003EE0B4242090003EE0B423067408
:103C100002900042F090003EE0B42406900042740E
:103C200001F090003E7401F0900074E0FE9000D727
:103C3000E02E900044F0900044E0D39424400B9098
:103C40000044E0C39424900044F0900044E0D394F6
:103C500024400B900044E0C39424900044F0900072
:103C600044E06403601F900044E064066017900025
:103C700044E06412600F900044E064156007900017
:103C800044E0B42406900044E004F0900044E06472
:103C900002601F900044E064056017900044E064F7
:103CA00011600F900044E064146007900044E0B499
:103CB0002306900044E014F0900044E0D3942440A4
:103CC0000B900044E0C39424900044F0900044E042
:103CD000D39412400D900044E0C39412900045F03C
:103CE000800A900044E02412900045F07551129033
:103CF00000BAE090003FF090003FE0B40206900070
:103D00003F7401F090003FE0B40306740490003F5C
:103D1000F090003FE0B41106741090003FF0900066
:103D20003FE0B41206741390003FF090003FE0B4FF
:103D30001406741390003FF090003FE0B415067431
:103D40001690003FF090003FE0B4230674229000EC
:103D50003FF090003FE0B42406742590003FF090BF
:103D6000003FE0B42606742590003FF090003FE04D
:103D7000B42706742890003FF090003FE0B4350669
:103D8000743490003FF090003FE0B43606743790F2
:103D9000003FF090003FE0B43806743790003FF0E9
:103DA00090003FE0B43906743A90003FF090003F35
:103DB000E0B44706744690003FF090003FE0B448FE
:103DC0000690003F7401F090003FE0D39424400F30
:103DD00090003FE0C3942490003FF0D21A8002C2CA
:103DE0001A90003FE0D39412400D90003FE0C3943E
:103DF00012900040F0800A90003FE02412900040B2
:103E0000F022C293C294C291C292C287C290E5B519
:103E100054EFF5B5E5B554DFF5B5C296C295C2A02D
:103E2000C297C2A2C2A1E5B554BFF5B5E5B5547FAE
:103E3000F5B5E5B554FBF5B5C209755E469000BD14
:103E4000E07005756D028003756D0375550075543E
:103E50000090000874FFF0A374DCF0C20EC211746D
:103E6000C8900035F074C8900039F0755300755251
:103E700000C204754600E56FB40903756F007563F1
:103E800000900017E4F0A3F0757010C20CC20DC2D0
:103E90000375570075560090000AE4F0A3F09000F7
:103EA0000CE4F0A3F0C22775590075580090007F0C
:103EB000E075F032A4FFAEF090001FEEF0A3EFF03B
:103EC00090006EE4F090006FE4F0C222D217C216A8
:103ED000D218C219C21AC21B22755B00755A00AEF5
:103EE0005AAF5B7402C39F74019E5003023F9790C8
:103EF000678B120048E493900073126ABA0FBF00F8
:103F0000010EE0FC90678B120048ECFEE493FFEE9C
:103F1000C39F5026AE5AAF5B0FBF00010E90678B58
:103F2000120048AE5AAF5BE493FC90678B120048D6
:103F3000E493900073126ABAECF0AE5AAF5B9067EC
:103F40008B120048E493900073126ABAE0FC906709
:103F50008D120048ECFCE493FDECD39D4019906772
:103F60008D120048E493FC90678B120048E4939014
:103F70000073126ABAECF0AE5AAF5B74022FFF50B6
:103F8000010E8E5A8F5B785B740126F6500418E49C
:103F900036F64003023EDF22755B00755A00AE5ACA
:103FA000AF5B7433BE00039F500302406590688D81
:103FB000120048E493900073126ABA0FBF00010E1A
:103FC000E0FC90688D120048ECFEE493FFEEC39F86
:103FD0005026AE5AAF5B0FBF00010E90688D1200E5
:103FE00048AE5AAF5BE493FC90688D120048E493AE
:103FF000900073126ABAECF0AE5AAF5B90688D1203
:104000000048E493900073126ABAE0FC90688F1243
:104010000048ECFCE493FDECD39D401990688F12AE
:104020000048E493FC90688D120048E4939000737C
:10403000126ABAECF0AE5AAF5B742D6F4E70067513
:104040005B33755A00AE5AAF5B74022FFF50010EFE
:104050008E5A8F5B785B740126F6500418E436F6AE
:104060004003023F9E22755B00755A00AE5AAF5B5B
:104070007433BE00039F50030241339068C01200A6
:1040800048E493900073126ABA0FBF00010EE0FC7F
:104090009068C0120048ECFEE493FFEEC39F5026E8
:1040A000AE5AAF5B0FBF00010E9068C0120048AE61
:1040B0005AAF5BE493FC9068C0120048E493900010
:1040C00073126ABAECF0AE5AAF5B9068C012004847
:1040D000E493900073126ABAE0FC9068C212004840
:1040E000ECFCE493FDECD39D40199068C2120048AB
:1040F000E493FC9068C0120048E493900073126A45
:10410000BAECF0AE5AAF5B742D6F4E7006755B3330
:10411000755A00AE5AAF5B74022FFF50010E8E5AD3
:104120008F5B785B740126F6500418E436F6400382
:1041300002406C22E50C90632AF82828730241FAA9
:1041400075E700A230B34008E5B54408F5B5800630
:10415000E5B554F7F5B575E7100241FA75E700A229
:1041600030B34008E5B54402F5B58006E5B554FD29
:10417000F5B575E7100241FAA23092A2807CA23018
:1041800092A1807675E700A230B34008E5B54440BF
:10419000F5B58006E5B554BFF5B575E710805B75DC
:1041A000E700A230B34008E5B54480F5B58006E5E8
:1041B000B5547FF5B575E7108040A2309287803AFC
:1041C000A2309290803475E700A230B34008E5B584
:1041D0004410F5B58006E5B554EFF5B575E71080E8
:1041E0001975E700A230B34008E5B54420F5B58065
:0A41F00006E5B554DFF5B575E710DC
:10632A0002413D02414002415C02417802417E0243
:10633A00418402419F0241BA0241C00241C6024160
:01634A00E171
:1041FA002285F97385FA747E017F00E574126A8953
:10420A00E5732FFF50010E8E5A8F5BAC5CAD5DEFEC
:10421A002DFDEE3CFC8C5C8D5DD293D294D291D272
:10422A0092E55DF5FBE55CF5FCE55DF5E9E55CF538
:10423A00EAE55DF5EBE55CF5ECE55DF5EDE55CF5EC
:10424A00EE2275A71085F97385FA747E017F00E561
:10425A0074126A89E5732FFF50010E8E5A8F5B7EA6
:10426A00017F769000F8E0126A89AC5AAD5BED2FB7
:10427A00FFEC3EFE8E5C8F5DE55DF5FDE55CF5FECF
:10428A00900062E4F075A7007412900047F022854E
:10429A00F97385FA747E017F00E574126A89E57301
:1042AA002FFF50010E8E5A8F5B900011E0FCA3E0A5
:1042BA00FDEF2DFDEE3CFC8C5C8D5DE55DF5FDE5CD
:1042CA005CF5FE220564229000BBE0B40353900023
:1042DA00D9E0B4012EA2D8B34004C293C287A2D9AE
:1042EA00B34004C294C290A2DAB34008C291E5B5C1
:1042FA0054EFF5B5A2DBB34008C292E5B554DFF539
:10430A00B5801CA2D8B34002C293A2D9B34002C25C
:10431A0094A2DAB34002C291A2DBB34002C29280F5
:10432A002EA2D8B34012C293C2919000D9E060087D
:10433A00C287E5B554EFF5B5A2D9B34012C294C20B
:10434A00929000D9E06008C290E5B554DFF5B5A2B5
:10435A00DCB34030A29650067419900047F0A2953B
:10436A0050067419900047F0A2A0500674199000E4
:10437A0047F0A29750067419900047F0C296C2956A
:10438A00C2A0C29775D8402285A77275A710A2D875
:10439A00B34002C287A2D9B34002C290A2DAB340A4
:1043AA0006E5B554EFF5B5A2DBB34006E5B554DF33
:1043BA00F5B5A2DCB340089000C7E0900062F07542
:1043CA00D8408572A72290F800E4936406600280C0
:1043DA00FE75B50075840175A70075FF8075EF0637
:1043EA00900043E4F075C91075A70F75A1C775A7AA
:1043FA000075D90075CE0C75A70F75F1FE75F2FF21
:10440A0075F30775F47875A4BA75A5FF75A60775CF
:10441A00AE0075AFFF75D48175D5FF75D6FF75D718
:10442A00FF75A70075A20175A14775F80975D8002F
:10443A0075D90475DA0975DB0975DC0975DD097545
:10444A00DE0975D84075A71075D80075D90475DAD4
:10445A000975DB0975DC0975DD0975DE0975D84052
:10446A0075A70075E60875E71075BC0175BE047579
:10447A00BD6C75BE0775BDA075BE0875BD0175BC5E
:10448A000075BB1875BC2075BA0875E88075D1131C
:10449A0075A70F75E10575E20075C740123E0275F2
:1044AA009700759780740A126A697597C0E59754E0
:1044BA0020700280F8758F0275A700D2AF75980038
:1044CA0075A90C75A70F75AB4375ADFB75AC1E7559
:1044DA00A71075C91875CA0075CB0075C80475A7E9
:1044EA0000758912758E04758C00758A00C2A9D26E
:1044FA008C758D00758B00D2ABD28E75B62075D9AE
:10450A0044C299C22674C8F5097508001200F875E4
:10451A00A70FE5FB900051F0E5FA900052F0E5F99B
:10452A00900053F075A70090F800E493F527120263
:10453A0017900886E0D394035007900886E0B401E8
:10454A00067400900886F074019000BCF09008860A
:10455A00E090634BF8282873802A802875A70F7586
:10456A00F30F75A700A2A3400674029000BCF08066
:10457A001375A70F75F31775A700A2A44006740256
:04458A009000BCF0F1
:0C634B0002456202456402456602457B83
:10458E009000BCE0B4022AC2251205B67402900057
:10459E00BCF0900886E0906357F82828738010804E
:0F45AE000E74009000CBF0800674009000D8F0DF
:0C6357000245AB0245AD0245AF0245B760
:1045BD008028D2251204D574019000BCF090088695
:1045CD00E0906363F82828738010800E74009000CB
:0A45DD00CBF0800674009000D8F0C7
:0C6363000245D50245D70245D90245E1AC
:1045E7001233109000C6E07006740A9000C6F0906F
:1045F70000A7E0700674E39000A7F09000ADE00418
:10460700900065F01235B490F807E493900058F0E5
:10461700900058E0440A900058F0900058E054FE8B
:10462700900058F07406900049F0740190004AF029
:1046370090F802E49390004BF0740390004CF074F0
:104647000590004DF0742D90004EF0740690004FC9
:10465700F090004BE0B40506740590004FF0740627
:10466700900050F090F804E493900054F074009098
:104677000055F090F805E493900056F090F806E4A2
:1046870093900057F074FF900059F0123ED99000B4
:104697004BE0B405051240668003123F989000E294
:1046A700E090005EF0900099E090005FF090009A33
:1046B700E0900060F0A2B6B39205A2B3B39206A24F
:1046C700A4B3921DA2A3B3921E90005AE4F0756F93
:1046D70000743A900773F074FD900774F090005BD4
:1046E700E4F0756E01900047E4F09000BDE0B4017E
:1046F70006741A900047F0C21C756300C20AD20BF9
:10470700C203757100C21F12009E755F00756B00B2
:1047170075610075653275660075670075680075A7
:104727006900756A00900017E4F0A3F0756C00D279
:10473700B2D2A4D2B0D2B1D2A3D2A7D2A6D2A5D296
:10474700B790007FE0D394FA400674FA90007FF0A8
:104757007E017F00900060E0126A8990005FE02F81
:10476700FF50010E900021EEF0A3EFF0EFD394FF7E
:10477700EE940F4007900021E4F0A3F090005EE074
:10478700700674FF90005EF09000BDE07005756DD7
:10479700028003756D039000BEE0D3940140067458
:1047A700009000BEF09000C4E0C3940A5006740A5B
:1047B7009000C4F09000CEE0700674019000CEF037
:1047C7009000CEE0B4FF0674FE9000CEF09000D5C6
:1047D700E0D394FE400674FE9000D5F09000FBE015
:1047E700D39402400674019000FBF0900111E0D3CE
:1047F700940140067401900111F074019000DBF000
:1048070074019000DCF074009000E3F074009000F5
:10481700FFF07400900103F074299006B9F0742A30
:104827009006BDF0D29C9000AEE0D394044006748D
:10483700049000AEF09000E0E0D3940440067404C6
:104847009000E0F0E570D394104003757010900667
:10485700BAE0D3940C400674009006BAF09006BEF6
:10486700E0D3940C400674009006BEF09006C2E0B8
:10487700D3940C400674009006C2F09006C6E0D3AD
:10488700940C400674009006C6F09006CAE0D394D4
:104897000C400674009006CAF09006CEE0D3940C44
:1048A700400674009006CEF09006D2E0D3940C40F8
:1048B7000674009006D2F09006D6E0D3940C40061A
:1048C70074009006D6F09006DAE0D3940C40067494
:1048D700009006DAF09006DEE0D3940C40067400F0
:1048E7009006DEF0D2EC75CF01A298B34005C298CE
:1048F700120697E54D6006A299B3B340028005C240
:1049070099120B78E54E64016005E54EB404028008
:10491700D5C28E7E107F00E564126A89E58D75F039
:1049270010A4FDACF0EF2DFDEE3CFCE58B75F0100F
:1049370084FF7E00ED2FFFEC3EFE8E548F55D28E06
:104947009000A0E060099000A0E0C3943D40028081
:104957005C900019126A97900019E0FEA3E0FF909F
:10496700001BE0FCA3E0FDEFB50542EEB5043EB247
:1049770014A204B3401975E700A214B34008E5B5C3
:104987004404F5B58006E5B554FBF5B575E7109019
:10499700001BE0FEA3E0FF90001DE0FCA3E0FDEF9D
:1049A7002DFDEE3CFC90001BECF0A3EDF09000AD6C
:1049B700E060099000ADE0C394034003024A671228
:1049C7002745A204B3500990005AE0C3941C400243
:1049D7008006900097E0F545E54575F002A4FFAE27
:1049E700F090087BEEF0A3EFF0900084E0C39561B0
:1049F7004007E55FC39560500790087BE4F0A3F09C
:104A070075E700AE2EAF2F90087BE0FCA3E0FDEF2B
:104A1700D39DEE9C4020E5B5547FF5B59000ADE001
:104A2700B402099000CBE0C3940240028006E5B5CA
:104A37004440F5B5802790005AE0C3942A501EE5FC
:104A4700B54480F5B59000ADE0B402099000CBE025
:104A5700C3940240028006E5B554BFF5B575E7106B
:104A67009000ADE0B4032A12286075E700AE2EAFC0
:104A77002F90087BE0FCA3E0FDEFD39DEE9C400860
:104A8700E5B54480F5B58006E5B5547FF5B575E71E
:104A970010900088E06009A2B3300601B3B340026A
:104AA7008056A2B3300601B3404EA2B3300801B31B
:104AB7004039A217403090006DE0D3955E402590B5
:104AC700006FE0701390006EE0B4010690006F7401
:104AD70001F090006EE004F0A216B3400590006E5E
:104AE700E4F0D216D217A208B39206A208B330B3E5
:104AF70001B34004A2089206A2B6300501B35003E1
:104B07000251FCA2B6300501B350030251FCA2B614
:104B1700300701B350030250A8756E009000A0E063
:104B2700B43D1975E700A207B34008E5B554FBF596
:104B3700B58006E5B54404F5B575E710055EA2092D
:104B4700B3B35013AE54AF55900008E0FCA3E0FD9B
:104B5700EDC39FEC9E4003024D4EE55EB4112175F7
:104B67005E13AE56AF57AC54AD55EF2DFDEE3CFC82
:104B770074028C068D071200398E568F57024D4CE2
:104B8700E56DB4032EA227B34022E55EB423037577
:104B97006D01E55EC3942350069000477401F0E56C
:104BA7005ED3942340067402900047F0755E01D2ED
:104BB700278062E56DB4020A756D01755E23C21622
:104BC700C218E55EB42305755E018049900047E091
:104BD7007034E55EC3942350069000477401F0E5F6
:104BE7005ED3942340067402900047F0E55EC394B9
:104BF700235002D21CE55ED394234002D21CC296F6
:104C0700C295C2A0C2979000BDE0B40105123E0252
:104C17008003755E01AE56AF57AC54AD55EF2DFD11
:104C2700EE3CFC74028C068D071200398E568F57A6
:104C37009000A0E060099000A0E0C3943D4002808E
:104C470049900019E0FEA3E0FF9000A0E08E048FDA
:104C570005FF126A7974018C068D071200399000DE
:104C67001DEEF0A3EFF090001DE0F8A3E090001B0D
:104C7700C8F0A3C8F0900019E4F0A3F0C21475E7D8
:104C870000E5B554FBF5B575E710A2A4B34002C221
:104C97001DA2A3B34002C21EA21CB34002C21CB293
:104CA7001990006FE0B40111A216B34004D2198025
:104CB70002C219740290006FF090006FE0C3940273
:104CC7005006A204B3B340028006740290006FF04E
:104CD7009000C9E0640460079000BBE0B4036290F1
:104CE7000088E0600690006FE07002800DA2183027
:104CF7001601B3400590006EE4F09000BDE064013A
:104D07006006A222B3B35017900088E06009A2168C
:104D1700301801B3B3400280067405900047F0B223
:104D270018A217B3401BA216B34004D2188002C2C0
:104D3700189000BDE0700690006FE070028002D20C
:104D470022C216C2178040E55E6414603AAE56AFC1
:104D570057AC54AD55EF2DFDEE3CFC74018C068D20
:104D6700071200398E568F57E56DC39402500DAC6C
:104D770054AD5574B6C39D740E9C40028009123E13
:104D8700027406900047F0E55EB4141E755E16AE19
:104D970056AF57AC54AD55EF2DFDEE3CFC74028C6D
:104DA700068D071200398E568F57E55EB4231274AD
:104DB70003900047F0D21C9000BDE0B40103123EFF
:104DC70002AE58AF59AC54AD55EF2DFDEE3CFC8CFF
:104DD700588D59AE54AF55EFD39DEE9C40119000BE
:104DE7000FE0FAA3E0FBEBC394E8EA9403400280E8
:104DF7000690000F126A9790000CE0FEA3E0FFAC4C
:104E070054AD55EF2DFDEE3CFC90000CECF0A3EDFE
:104E1700F09000BDE0B40118AE54AF557405126AA6
:104E2700897401120039900008EEF0A3EFF08011A9
:104E3700AE54AF557402126A89900008EEF0A3EFE2
:104E4700F0C28E758D00758B007564007555017500
:104E57005400D28EE55E240875F00984AFF07E0019
:104E6700EF4E6003024EF0E56D6013AE56AF577418
:104E770009126A8990000AEEF0A3EFF0800F900004
:104E87000CE0F8A3E090000AC8F0A3C8F090000A6D
:104E9700E0FEA3E0FFEF4E600B7C797DB5126977EA
:104EA7008E528F5390000CE4F0A3F0AE52AF5374C0
:104EB70028BE00039F5010E5632FFF50010E7401B9
:104EC7001200398E528F538553639000C4E0A85265
:104ED700B8000DD395534008E553900046F080097C
:104EE7009000C4E014900046F09000BBE0B40308C3
:104EF70090003FE0655E6002800EA219301A01B390
:104F07004004D21B8002C21BE55E640B6005E55EB0
:104F1700B41D099000ADE06003122411900044E035
:104F2700655E6007900045E0B55E03756F00A20AF5
:104F3700B35006A209B3B34003024FE8900079E0EB
:104F4700B401739000FBE0B40214120D19900063D2
:104F5700E075F0BEA4FFAEF08E5C8F5D8056E5670E
:104F670075F00A84FF7E00900573120048E0F55B38
:104F7700755A00AE5AAF5B90009EE0126A8974645E
:104F87008E048F05FF126A798C5C8D5DE55D90005C
:104F97000EF0AE5AAF5B900077E0126A8974648EA8
:104FA700048F05FF126A7974BE8C068D07126A8911
:104FB7008E5C8F5D8017900077E075F0BEA4FFAE22
:104FC700F08E5C8F5D90009EE090000EF0E561C36F
:104FD70094CC5006E55D455C700280031241FBD21C
:104FE7000AE56DB40106E55E640B60028018900067
:104FF700C9E0B40405757003800975700190004815
:105007007401F0756D00E56D60030250A39000C058
:10501700E0600D900062E0A852B800069553400288
:1050270080389000C0E0B4021790003DE0655E60F4
:105037000790003EE0B55E03757003756C00800C49
:10504700C201756C00900017E4F0A3F0900062E0D5
:1050570060067409900047F0804290003DE0655E6D
:10506700600790003EE0B55E339000C9E0B4040FDE
:10507700A222B34005757001800375700380037524
:10508700700190003DE0B55E069000487401F09015
:10509700003EE0B55E067402900048F0A207B392A6
:1050A70005A207B330B601B350030251FC756E0178
:1050B7009000A0E0B43D1975E700A207B34008E5EA
:1050C700B54404F5B58006E5B554FBF5B575E710AD
:1050D700A226400575FFA0D22675E700E5B5440175
:1050E700F5B575E710741C90005AF0A2079205E514
:1050F7005ED3944A4014D209E55ED3946D400B7495
:1051070004900047F0D21C755E469000C8E0B401D9
:1051170007E56AC3941440028009123E0274139093
:105127000047F0E56AC394415009740E900047F0B8
:10513700123E0290004FE0FE90004BE0C39E4009F4
:1051470090004BE0D39408400974FB900047F0129D
:105157003E02900054E06015900054E0FE90004E2F
:10516700E06E600974FE900047F0123E02900886D8
:10517700E060069000F8E06002807A74019000BC5D
:10518700F0900886E090636FF828287380188016DF
:10519700A2A3400674029000BCF0800AA2A44006B5
:0651A70074029000BCF050
:0C636F000251930251950251970251A374
:1051AD009000BCE0B40105A225B340028019D225C0
:1051BD00123E021204D574019000BCF0123310D2CD
:1051CD001F741B900047F09000BCE0B40206A225AE
:1051DD00B3B340028019C225123E021205B6740205
:1051ED009000BCF0123310D21F741B900047F0A238
:1051FD001CB34008C296C295C2A0C2979000F8E0B9
:10520D00600CAE52AF537414BE00059F4002803740
:10521D00900080E090637BF8282873802A8028A274
:10522D00A3B35005A21EB34002800512424CD21EFC
:10523D008015A2A4B35005A21DB3400280051242F1
:07524D004CD21D800280001D
:10637B0002522802522A02522C02523F025252025D
:02638B0052546A
:10525400A20CB3B3500890003FE0655E60030254B3
:105264008DA202B35006A201B3B340030254899045
:1052740000BBE0B40302800302544890006FE0B422
:105284000202800302542FA21BB3500302535C1288
:10529400345390010CE0601F900015E0FEA3E0FF82
:1052A400900104E0126A8974C88E048F05FF126AA3
:1052B400798C5C8D5D800A900015E0F55CA3E0F5C7
:1052C4005DAE5CAF5D745E126A8974058E048F05F1
:1052D400FF126A79AE5AAF5BED2FFFEC3EFE8E5C97
:1052E4008F5DE55DF5FBE55CF5FCD293A203B3406D
:1052F40002D2879000D9E0B4025B12348090010C92
:10530400E0D39404401BAE2CAF2D900108E0126A48
:105314008974C88E048F05FF126A798C5C8D5D8058
:1053240006852C5C852D5DAE5CAF5D745E126A896A
:1053340074058E048F05FF126A79AE5AAF5BED2FA8
:10534400FFEC3EFE8E5C8F5DE55DF5FBE55CF5FCF8
:1053540075A700D28702542D12345390010CE0D368
:105364009403401F900015E0FEA3E0FF900106E0C7
:10537400126A8974C88E048F05FF126A798C5C8D59
:105384005D800A900015E0F55CA3E0F55DAE5CAFCE
:105394005D745E126A8974058E048F05FF126A7942
:1053A400AE5AAF5BED2FFFEC3EFE8E5C8F5DE55D8C
:1053B400F5EBE55CF5ECD291A203B34006E5B54408
:1053C40010F5B59000D9E0B4025F12348090010C5E
:1053D400E0D39406401BAE2CAF2D90010AE0126A74
:1053E4008974C88E048F05FF126A798C5C8D5D8088
:1053F40006852C5C852D5DAE5CAF5D745E126A899A
:1054040074058E048F05FF126A79AE5AAF5BED2FD7
:10541400FFEC3EFE8E5C8F5DE55DF5EBE55CF5EC47
:1054240075A700E5B54410F5B58017123453E55D52
:10543400F5FBE55CF5FCE55DF5EBE55CF5ECD2939D
:10544400D2918041123453E55DF5FBE55CF5FCD265
:1054540093D291A203B34008D287E5B54410F5B5C1
:105464009000D9E0B4021E123480E55DF5FBE55CE2
:10547400F5FCE55DF5EBE55CF5EC75A700D287E599
:10548400B54410F5B5C20CD20DA20DB3B3500890BB
:105494000040E0655E60030256C9A202B35006A252
:1054A40001B3B340030256C59000BBE0B4030280CD
:1054B4000302568490006FE0B40202800302566B2C
:1054C400A21BB3500302559812345390010CE0D33D
:1054D4009401401F900015E0FEA3E0FF900105E059
:1054E400126A8974C88E048F05FF126A798C5C8DE8
:1054F4005D800A900015E0F55CA3E0F55DAE5CAF5D
:105504005D745E126A8974058E048F05FF126A79D0
:10551400AE5AAF5BED2FFFEC3EFE8E5C8F5DE55D1A
:10552400F5E9E55CF5EAD294A203B34002D2909087
:1055340000D9E0B4025B12348090010CE0D39405EE
:10554400401BAE2CAF2D900109E0126A8974C88EFD
:10555400048F05FF126A798C5C8D5D8006852C5C56
:10556400852D5DAE5CAF5D745E126A8974058E0430
:105574008F05FF126A79AE5AAF5BED2FFFEC3EFE4A
:105584008E5C8F5DE55DF5E9E55CF5EA75A700D213
:105594009002566912345390010CE0D39403401FD7
:1055A400900015E0FEA3E0FF900107E0126A897401
:1055B400C88E048F05FF126A798C5C8D5D800A9019
:1055C4000015E0F55CA3E0F55DAE5CAF5D745E12C2
:1055D4006A8974058E048F05FF126A79AE5AAF5B2F
:1055E400ED2FFFEC3EFE8E5C8F5DE55DF5EDE55C39
:1055F400F5EED292A203B34006E5B54420F5B5908A
:1056040000D9E0B4025F12348090010CE0D3940717
:10561400401BAE2CAF2D90010BE0126A8974C88E2A
:10562400048F05FF126A798C5C8D5D8006852C5C85
:10563400852D5DAE5CAF5D745E126A8974058E045F
:105644008F05FF126A79AE5AAF5BED2FFFEC3EFE79
:105654008E5C8F5DE55DF5EDE55CF5EE75A700E527
:10566400B54420F5B58017123453E55DF5E9E55CE2
:10567400F5EAE55DF5EDE55CF5EED294D292804174
:10568400123453E55DF5E9E55CF5EAD294D292A2D1
:1056940003B34008D290E5B54420F5B59000D9E0B5
:1056A400B4021E123480E55DF5E9E55CF5EAE55DDA
:1056B400F5EDE55CF5EE75A700D290E5B54420F56F
:1056C400B5D20CC20DE57090638DF8282873025B87
:0556D400269000E0E05B
:06638D000256D20256D5B3
:1056D900906408F8282873121DB38012121DB38034
:0E56E9000D121E3D8008121EE98003121EE9FC
:0F6408000256E00256E50256EA0256EF0256F43B
:1056F700757002025B2612201512212C1224469087
:105707000873E0FEA3E0FF740A126A8990000AE0BA
:10571700FCA3E0FD74098F02FF126A798D078C03E1
:105727008E048A058B06126977900877EEF0A3EF4F
:10573700F09000C9E0B401087478BE00059F4002EC
:10574700800D7478900877F8E4F0E8A3F0801B9058
:105757000877E0FEA3E0FF74F0BE00039F500B74D0
:10576700F0900877F8E4F0E8A3F0E53670037536B3
:1057770001900877E0FEA3E0FFE5362FFF50010E0A
:0F578700900877EEF0A3EFF0757003900048E004
:036393000256FDB2
:10579600906417F82828738010A22F400375700AAA
:0957A6008007A22F400375700B6F
:0964170002579D02579F0257A88D
:1057AF00025B269006BAE060077401F50812256DBA
:1057BF009000F9E0B401149000FAE0A852B8000488
:1057CF0095535007E55FC3956040028009741590AB
:1057DF000047F00258669000AEE0D39402403F902D
:1057EF000082E02403A852B800049553500990009A
:1057FF0084E0D3956150028008D20274089000476C
:10580F00F0900082E0A852B80005D39553500B904A
:10581F000084E02403C395615002C20280399000D6
:10582F0082E02403A852B8000495535007E55FC3E4
:10583F00956040028008D2027408900047F09000F3
:10584F0082E0A852B80005D395535009E560240FA4
:10585F00C3955F5002C2029000C8E07007E56AC3AB
:10586F00941440028002D2029000BDE0B40102D233
:10587F0002A2024005757004800A7570109000171F
:0B588F00E4F0A3F0025B269000AEE006
:066396000257B202589606
:10589A00906420F8282873120E038012120E0380D7
:0E58AA000D120FB180081210638003121063FC
:0F6420000258A10258A60258AB0258B00258B554
:1058B8009006BEE0600675080212256D7570050237
:1058C8005B261211A37570069006C2E06006750883
:1058D8000312256D9006C6E0600675080412256D52
:1058E800025B2690000EE06006A204B3B34002807B
:1058F8001D90000EE02529FFAE2850010E8E288F3E
:1059080029E55ED39412500690000EE014F01213AD
:10591800E97570079006CAE0600675080512256DDE
:105928009006CEE0600675080612256D025B26908B
:1059380000FBE0B40203120D91121819757008905B
:1059480006D2E0600675080712256D9006D6E0605D
:105958000675080812256D025B26121BD5A20CB32A
:105968005005A20DB340028004D20CD20D75701000
:105978009006DAE060077409F50812256D9006DED6
:10598800E06007740AF50812256D025B26025B26A3
:10599800900037E0C39446500AC296C2A07446905D
:1059A8000037F0900041E0B4011DE536240AF536D1
:1059B800900877E0FEA3E0FF740A2FFF50010E90D5
:1059C8000877EEF0A3EFF0900041E0B4021DE53651
:1059D8002414F536900877E0FEA3E0FF74142FFF37
:1059E80050010E900877EEF0A3EFF085365B755AFC
:1059F8000090003DE0F5731234CBE55D900037F080
:105A0800900004E55AF0A3E55BF0E573900038F0E8
:105A1800C20F900877E0F55AA3E0F55B90003DE0EF
:105A2800F5731234CBE55D900035F0900000E55A2F
:105A3800F0A3E55BF0E573900036F0A200921090B9
:105A48000041E06002B210C20E757003025B26903E
:105A5800003BE0C3944650139000C9E0B40102C271
:105A680096C295C297744690003BF0900042E0B40D
:105A7800011DE536240AF536900877E0FEA3E0FF1D
:105A8800740A2FFF50010E900877EEF0A3EFF09004
:105A98000042E0B4021DE5362414F536900877E09C
:105AA800FEA3E0FF74142FFF50010E900877EEF06C
:105AB800A3EFF085365B755A0090003EE0F573124F
:105AC80034CBE55D90003BF0900006E55AF0A3E585
:105AD8005BF0E57390003CF0C212900877E0F55A4D
:105AE800A3E0F55B90003EE0F5731234CBE55D90E2
:105AF8000039F0900002E55AF0A3E55BF0E57390F9
:105B0800003AF0A2009213900042E06002B213C281
:0E5B18001175700380088006800480028000F2
:10639C000258CA0258EB0259370259620259950247
:1063AC005998025A57025B1E025B20025B22025B69
:0463BC0024025B2636
:105B2600900035E0B55E028003025C03A20E40726F
:105B3600900000E0FEA3E0FFEF4E6021AE56AF57A7
:105B4600900000E0FCA3E0FD120003740A8E048FAF
:105B560005FF126A79900000ECF0A3EDF090003694
:105B6600E0601A900000E0FEA3E0FFAC56AD57EFF0
:105B76002DFDEE3CFC900000ECF0A3EDF09000361D
:105B8600E0D39401401A900000E0FEA3E0FFAC567B
:105B9600AD57EF2DFDEE3CFC900000ECF0A3EDF0D0
:105BA600D20EAE54AF55900000E0FCA3E0FDEFC36B
:105BB6009DEE9C40481242999000C9E09063C0F85F
:105BC6002828738030D296802CD2968028D296D2FE
:105BD600A08022A2104010A223301801B34004D2A4
:105BE600A08002D296800EA223301801B34004D2C0
:055BF600968002D2A020
:0F63C000025BC9025BCB025BCF025BD3025BD9EE
:105BFB00C20E74C8900035F0A20EB3B350079000DC
:105C0B0035E0B55E0280481242999000C9E090637E
:105C1B00CFF82828738030D296802CD2968028D249
:105C2B0096D2A08022A2104010A223301801B340BC
:105C3B0004D2A08002D296800EA223301801B3406A
:075C4B0004D2968002D2A0F2
:0F63CF00025C20025C22025C26025C2A025C3027
:105C520074C8900035F0C20E900037E0B55E028045
:105C620003025CFBA20F4072900004E0FEA3E0FF7F
:105C7200EF4E6021AE56AF57900004E0FCA3E0FD6A
:105C8200120003740A8E048F05FF126A79900004D1
:105C9200ECF0A3EDF0900038E0601A900004E0FE12
:105CA200A3E0FFAC56AD57EF2DFDEE3CFC90000497
:105CB200ECF0A3EDF0900038E0D39401401A90008C
:105CC20004E0FEA3E0FFAC56AD57EF2DFDEE3CFC29
:105CD200900004ECF0A3EDF0D20FAE54AF5590005B
:105CE20004E0FCA3E0FDEFC39DEE9C400CC296C213
:105CF200A07446900037F0C20FA20FB3B3500790C2
:105D02000037E0B55E02800CC296C2A074469000D5
:105D120037F0C20F900039E0B55E028003025DF3F6
:105D2200A2114072900002E0FEA3E0FFEF4E60215C
:105D3200AE56AF57900002E0FCA3E0FD12000374E0
:105D42000A8E048F05FF126A79900002ECF0A3ED2F
:105D5200F090003AE0601A900002E0FEA3E0FFAC8F
:105D620056AD57EF2DFDEE3CFC900002ECF0A3ED9A
:105D7200F090003AE0D39401401A900002E0FEA3B2
:105D8200E0FFAC56AD57EF2DFDEE3CFC900002EC6F
:105D9200F0A3EDF0D211AE54AF55900002E0FCA397
:105DA200E0FDEFC39DEE9C40481242999000C9E08D
:105DB2009063DEF82828738030D296802CD29580AA
:105DC20028D295D2978022A2134010A22430180123
:105DD200B34004D2978002D295800EA224301801DB
:095DE200B34004D2958002D2976F
:0F63DE00025DB9025DBB025DBF025DC3025DC916
:105DEB00C21174C8900039F0A211B3B350079000E0
:105DFB0039E0B55E0280481242999000C9E0906389
:105E0B00EDF82828738030D296802CD2958028D23A
:105E1B0095D2978022A2134010A224301801B340D0
:105E2B0004D2978002D295800EA224301801B34081
:075E3B0004D2958002D2970A
:0F63ED00025E10025E12025E16025E1A025E204F
:105E420074C8900039F0C21190003BE0B55E028048
:105E520003025EF4A2124072900006E0FEA3E0FF8D
:105E6200EF4E6021AE56AF57900006E0FCA3E0FD76
:105E7200120003740A8E048F05FF126A79900006DD
:105E8200ECF0A3EDF090003CE0601A900006E0FE1A
:105E9200A3E0FFAC56AD57EF2DFDEE3CFC900006A3
:105EA200ECF0A3EDF090003CE0D39401401A900096
:105EB20006E0FEA3E0FFAC56AD57EF2DFDEE3CFC35
:105EC200900006ECF0A3EDF0D212AE54AF55900064
:105ED20006E0FCA3E0FDEFC39DEE9C40159000C9D7
:105EE200E0B40102C296C295C297744690003BF09C
:105EF200C212A212B3B3500790003BE0B55E02801B
:105F0200159000C9E0B40102C296C295C2977446C8
:105F120090003BF0C2129000CBE0B4020280030278
:105F2200604C90005CE0D39566506490005CE0F4B5
:105F3200042566FE9000CEE08E00F5F0E884FF7E38
:105F4200008F73EFC39410500CEF8573F0A4FDAC77
:105F5200F08D7380037573FF90005CE0D3957340FE
:105F62000B90005CE0C39573F5718003757100902E
:105F720000E9E0D3957140069000E9E0F5719000E8
:105F8200EAE0C3957150069000EAE0F571807190E5
:105F9200005CE0C39566FE9000CEE08E00F5F0E86E
:105FA20084FF7E008F73EFC39410500CEF8573F063
:105FB200A4FDACF08D7380037573FF85735B755A16
:105FC2000090005CE0255BFFAE5A50010E8E5A8FA6
:105FD2005B74FFBE0009D39F4005855B718003752A
:105FE20071FF9000E9E0D3957140069000E9E0F579
:105FF200719000EAE0C3957150069000EAE0F571F5
:10600200A204B3B3500D90005DE0FE9000D6E0D341
:106012009E500280147407900047F075E700E5B5C2
:1060220054BFF5B575E710802175A71075E700E537
:10603200CDC395714008E5B554BFF5B58006E5B509
:106042004440F5B575E71075A7009000E6E0604E94
:106052009000F0E0A852B80004955350179000EF5A
:10606200E0A852B8000ED3955340099000F1E0D356
:1060720095614002801575A710E5CDC394BF400419
:10608200C2A28002D2A275A700801375A710E5CD27
:10609200C394404004C2A28002D2A275A70090001D
:1060A200E7E0604E9000F3E0A852B8000495535028
:1060B200179000F2E0A852B8000ED3955340099011
:1060C20000F4E0D395614002801575A710E5CDC3B9
:1060D20094BF4004C2A18002D2A175A700801375AB
:1060E200A710E5CDC394404004C2A18002D2A1759D
:1060F200A700E56FC39409500AA2EDB34005C2EDB3
:10610200122A07AE54AF557498C39F743A9E400C3E
:1061120090005BE0C3945A4003026327A209B34094
:1061220009123E027406900047F0A20BB3500EE52E
:1061320061D394334007E561C394CC4002804A9016
:1061420000FBE0B40214120D19900063E075F050E8
:10615200A4FFAEF08E5C8F5D800F900077E075F04B
:1061620050A4FFAEF08E5C8F5DE55D455C601AA2C7
:1061720026400575FFA0D226E5B54401F5B5741C8D
:1061820090005AF01241FBD20B90005BE0D39401D5
:106192004007E561C3941A40028002C20B9006BA1E
:1061A200E060077401F50812256D9006BEE06007F5
:1061B2007402F50812256D9006C2E060077403F5BB
:1061C2000812256D9006C6E0600675080412256D5A
:1061D2009006CAE0600675080512256D9006CEE0AD
:1061E200600675080612256D9006D2E060067508F5
:1061F2000712256D9006D6E0600675080812256D17
:106202009006DAE0600675080912256D9006DEE058
:10621200600675080A12256D90005BE0C3945A501F
:1062220026E56FB4090990005BE004F0756F0090F9
:10623200005BE0B45A0FA226400575FFA0D226E506
:10624200B54401F5B5803BE56FB40903756F007580
:106252005500755400758D00758B007564009000B3
:106262005AE0C3942A500890005AE004F080067461
:106272002A90005AF090005AE0B42A06E5B554FE7E
:10628200F5B590005BE0D394014007E56AC3944101
:1062920040028009740E900047F0123E0290088678
:1062A200E060069000F8E06002807A74019000BC21
:1062B200F0900886E09063FCF82828738018801616
:1062C200A2A3400674029000BCF0800AA2A4400679
:0662D20074029000BCF014
:0C63FC000262BE0262C00262C20262CEF7
:1062D8009000BCE0B40105A225B340028019D22584
:1062E800123E021204D574019000BCF0123310D291
:1062F8001F741B900047F09000BCE0B40206A22572
:10630800B3B340028019C225123E021205B67402C8
:106318009000BCF0123310D21F741B900047F0029B
:0263280048ED3E
:10642F000000010001400160018001A001C001E0F6
:10643F0002000300039603B603D603F4040005001D
:10644F000512052405360548055A056C057E05908D
:10645F0005A805C005DE0600061406280646066ECA
:10646F0006AE05CF00FF013F015F017F019F01BF16
:10647F0001DF01FF02FF039503B503D503F303FF0C
:10648F0004FF05110523053505470559056B057DE6
:10649F00058F05A705BF05CE05F10613062706458F
:1064AF00066D06AD06ED05DD0FAA0FA50F9F0F9A1E
:1064BF000F940F8D0F870F800F780F710F680F607C
:1064CF000F570F4E0F450F3B0F300F250F1A0F0EA3
:1064DF000F020EF50EE80EDB0ECC0EBE0EAE0E9FAB
:1064EF000E8E0E7D0E6C0E5A0E470E340E200E0CB5
:1064FF000DF70DE20DCB0DB50D9D0D850D6D0D54E9
:10650F000D3A0D200D050CE90CCE0CB10C940C7648
:10651F000C580C3A0C1B0BFB0BDB0BBB0B9A0B79C0
:10652F000B570B350B130AF10ACE0AAB0A870A6415
:10653F000A400A1C09F809D409B0098C09670943F4
:10654F00091F08FB08D608B2088E086A08460823F8
:10655F0007FF07DC07B9079607730751072F070DCA
:10656F0006EC06CA06AA068906690649062A060A1D
:10657F0005EC05CD05B0059205750558053C0520C0
:10658F00050504EA04CF04B5049C04820469045190
:10659F0004390422040B03F403DE03C803B2039D82
:1065AF00038903750361034D033B0328031603049B
:1065BF0002F202E102D102C002B002A002910282F5
:1065CF000273026502570249023C022F0222021691
:1065DF00020901FD01F201E601DB01D001C601BB99
:1065EF0001B101A7019D0194018B01820179017015
:1065FF000168016001580150014801410139013220
:10660F00012B0125011E01180111010B010500FFCE
:10661F0000FA0FA60FA00F990F920F8B0F840F7C0C
:10662F000F740F6B0F620F580F4E0F430F380F2C55
:10663F000F1F0F120F050EF70EE80ED80EC80EB76C
:10664F000EA50E930E800E6C0E580E420E2C0E15CC
:10665F000DFD0DE40DCB0DB10D950D790D5D0D3FBC
:10666F000D200D010CE10CC00C9E0C7C0C590C354F
:10667F000C100BEA0BC40B9E0B760B4F0B260AFD6F
:10668F000AD40AAA0A800A550A2A09FF09D409A8B6
:10669F00097C0950092508F908CD08A10875084A91
:1066AF00081E07F307C8079D07730749072006F75A
:1066BF0006CE06A6067E06570630060A05E405BF77
:1066CF00059B057705540532051004EF04CE04AE83
:1066DF00048F047104530435041903FD03E203C747
:1066EF0003AD0394037B0363034B0334031E0308BF
:1066FF0002F302DE02CA02B602A30291027F026D0A
:10670F00025C024C023C022C021D020E020001F23E
:10671F0001E401D701CA01BE01B101A6019A018F9F
:10672F000185017A01700166015D0153014A014142
:10673F00013901310129012101190112010B010454
:10674F0000FD00F700F000EA00E400DE00D900D3FE
:10675F0000CE00C900C400BF00BA00B500B100AD43
:10676F0000A800A400A0009C009900950091008E45
:0C677F00008A008700840081007E007BFF
:10009E0075470090087DE4F0A3F0753100753000CF
:1000AE00754D00754E00C22AD22C900886E0600273
:1000BE00D21F74FE90087FF8E4F0E8A3F074FE906F
:1000CE000883F8E4F0E8A3F074FE900881F8E4F0F9
:1000DE00E8A3F0745A9008A5F0745A9008A6F0D2CE
:1000EE002DC228C22FC22EC22922750B00750A00FE
:1000FE00AE0AAF0BAC08AD09EDC39FEC9E40167473
:10010E00FF126A6975CF01780B740126F650041838
:10011E00E436F650DB22C2AF75D904758F0375B77E
:10012E00A575B7F190F800E4F0758F0175B7A57558
:10013E00B7F1E52790F800F075B7A575B7F190F80F
:10014E0001E4F075B7A575B7F1900899E090F80243
:10015E00F075B7A575B7F190089DE090F803F075AE
:10016E00B7A575B7F190089AE090F804F075B7A5A9
:10017E0075B7F190089BE090F805F075B7A575B7C7
:10018E00F190089CE090F806F075B7A575B7F19060
:10019E00089EE090F807F0758F0075D944D2AF2213
:1001AE00900043E0B4AB61C2AF75D90475B6227549
:1001BE00F522758F0375B7A575B7F1740090F6002B
:1001CE00F0758F01755B00755A00AE5AAF5B7413F4
:1001DE00BE00279F402475B7A575B7F1900885120C
:1001EE000048E0FC90F600120048ECF0785B7401D9
:1001FE0026F6500418E436F650D0758F0075F511BA
:10020E0075B62075D944D2AF22C2AF75F52275D915
:10021E0004755B00755A00AE5AAF5B7413BE0022B4
:10022E009F401F90F600120048E493FC9008851240
:10023E000048ECF0785B740126F6500418E436F6AC
:10024E0050D575D94475F511D2AF22900043E0B464
:10025E00AA028003020396C2AF75D90475B6227541
:10026E00F522758F0375B7A575B7F1740090EE0082
:10027E00F075B7A575B7F1740090F000F075B7A5DD
:10028E0075B7F1740090F200F075B7A575B7F174FB
:10029E000090F400F0758F01755B00755A00AE5A30
:1002AE00AF5B74FFC39F74019E402475B7A575B7ED
:1002BE00F1900073120048E0FC90EE00120048EC42
:1002CE00F0785B740126F6500418E436F650CF75BC
:1002DE005B00755A00AE5AAF5B74FFC39F74019EEC
:1002EE00402475B7A575B7F1900273120048E0FC73
:1002FE0090F000120048ECF0785B740126F6500482
:10030E0018E436F650CF755B00755A00AE5AAF5BE7
:10031E0074FFC39F74019E402475B7A575B7F19005
:10032E000473120048E0FC90F200120048ECF078E2
:10033E005B740126F6500418E436F650CF755B0058
:10034E00755A00AE5AAF5B74FFC39F74019E402472
:10035E0075B7A575B7F1900673120048E0FC90F4DE
:10036E0000120048ECF0785B740126F6500418E495
:10037E0036F650CF758F0075F51175B62075D944C8
:10038E00D2AF743A900773F022900043E0B4AA0201
:10039E0080030204D4C2AF75D90475B62275F52256
:1003AE00758F0375B7A575B7F1740090E600F075FB
:1003BE00B7A575B7F1740090E800F075B7A575B7DD
:1003CE00F1740090EA00F075B7A575B7F17400905E
:1003DE00EC00F0758F01755B00755A00AE5AAF5B7D
:1003EE0074FFC39F74019E402475B7A575B7F19035
:1003FE000073120048E0FC90E600120048ECF07822
:10040E005B740126F6500418E436F650CF755B0087
:10041E00755A00AE5AAF5B74FFC39F74019E4024A1
:10042E0075B7A575B7F1900273120048E0FC90E81D
:10043E0000120048ECF0785B740126F6500418E4C4
:10044E0036F650CF755B00755A00AE5AAF5B74FF2F
:10045E00C39F74019E402475B7A575B7F1900473C0
:10046E00120048E0FC90EA00120048ECF0785B7451
:10047E000126F6500418E436F650CF755B00755A17
:10048E0000AE5AAF5B74FFC39F74019E402475B7D4
:10049E00A575B7F1900673120048E0FC90EC0012BF
:1004AE000048ECF0785B740126F6500418E436F63A
:1004BE0050CF758F0075F51175B62075D944D2AF32
:1004CE00743A900773F022C2AF75D90475F5227590
:1004DE005B00755A00AE5AAF5B74FFC39F74019EEA
:1004EE00401F90EE00120048E493FC90007312003F
:1004FE0048ECF0785B740126F6500418E436F6509A
:10050E00D4755B00755A00AE5AAF5B74FFC39F740F
:10051E00019E401F90F000120048E493FC9002737D
:10052E00120048ECF0785B740126F6500418E4369D
:10053E00F650D4755B00755A00AE5AAF5B74FFC3AC
:10054E009F74019E401F90F200120048E493FC90AD
:10055E000473120048ECF0785B740126F650041810
:10056E00E436F650D4755B00755A00AE5AAF5B7424
:10057E00FFC39F74019E401F90F400120048E49345
:10058E00FC900673120048ECF0785B740126F6506E
:10059E000418E436F650D475F51175D944D2AF74FB
:1005AE003A900773F0C22B22C2AF75D90475F522AB
:1005BE00755B00755A00AE5AAF5B74FFC39F740132
:1005CE009E401F90E600120048E493FC90007312C8
:1005DE000048ECF0785B740126F6500418E436F609
:1005EE0050D4755B00755A00AE5AAF5B74FFC39F53
:1005FE0074019E401F90E800120048E493FC9002A4
:10060E0073120048ECF0785B740126F6500418E47F
:10061E0036F650D4755B00755A00AE5AAF5B74FF58
:10062E00C39F74019E401F90EA00120048E493FCA1
:10063E00900473120048ECF0785B740126F65004B7
:10064E0018E436F650D4755B00755A00AE5AAF5B9F
:10065E0074FFC39F74019E401F90EC00120048E48B
:10066E0093FC900673120048ECF0785B740126F64A
:10067E00500418E436F650D475F51175D944D2AF3E
:10068E00743A900773F0D22B22E54E64046006E5AF
:10069E009964FF60028031A22A4004D22A8027E5A5
:1006AE004E600874E6254E900047F0E54D600874E4
:1006BE00F0254D900047F0E54EB4010280FE754ED8
:1006CE0000754D00C22A8002C22AE54E903280F893
:1006DE00282873754E00E599B4FF03754D01E59911
:1006EE00B4FE03754D02E599B4FD03754D03E5990E
:1006FE00B4FC03754D04E599B4FA03754D05E599FF
:10070E00B4FB06754E01123E02E599B4F906754E1C
:10071E0004123E02E599D394E54007E599C394F09F
:10072E004002801685994F754E027E017F00E54F7F
:10073E00C394E6126A898E328F3390087DE4F0A35B
:10074E00F0E599D394C44007E599C394E64002803E
:10075E002885994F754E0374E5C3954FF533753261
:10076E0000AE32AF3390642F126A58E493F87401DE
:10077E009390087DC8F0A3C8F0D299020B77900829
:10078E0085E0700AA220B35005A221B34002804238
:10079E0090087DE0FEA3E0FF74FFBE00039F5009AA
:1007AE00EFC39446EE9406401190087DE0FEA3E060
:1007BE00FFEFD3946DEE9406401390087DE0FEA3F8
:1007CE00E0FF900073120048E599F080038599745C
:1007DE00801190087DE0FEA3E0FF900073120048A8
:1007EE00E599F090087D126A9790087DE0FEA3E0EF
:1007FE00FFEFB40106EEB407028003020970900702
:10080E0073E0B43C028003020970A220B35005A22B
:10081E0021B340030208E7C29C900885E0900111C5
:10082E00F0900886E0900080F0900887E09000A09D
:10083E00F0900888E09000C9F0900889E09000756B
:10084E00F090088AE09000BBF090088BE09000D901
:10085E00F090088CE09000ADF090088DE09000CB09
:10086E00F090088EE09000FBF090088FE090015F12
:10087E00F0900890E0900160F0900891E090016196
:10088E00F01235B490005EE09000E2F090005FE070
:10089E00900099F0900060E090009AF074AB900098
:1008AE0043F01201AE74AA900043F0A22BB34005A0
:1008BE001203978003120259900043E4F090015FF7
:1008CE00E0700C900160E07006900161E0600280C3
:1008DE0004C2208002D220807EC29C900111E09042
:1008EE000885F0900080E0900886F09000A0E090DF
:1008FE000887F09000C9E0900888F0900075E090AD
:10090E000889F09000BBE090088AF09000D9E09042
:10091E00088BF09000ADE090088CF09000CBE0904A
:10092E00088DF09000FBE090088EF0740090088F18
:10093E00F07400900890F07400900891F074AB90F1
:10094E000043F01201AE74AA900043F01202591245
:10095E0003977599FB80FED29C754E00754D007500
:10096E0099FB020B7790087DE0FEA3E0FFEF4E703F
:10097E000685993175300090087DE0FEA3E0FF7486
:10098E00016F4E701BAC30AD31AA32AB33ED2BFB89
:10099E00EC3AFA8A068B07900073120048E599F03C
:1009AE0090087D126A9790087DE0FEA3E0FF740226
:1009BE006F4E7021AC30AD3174566D4C7006E54FF4
:1009CE0064E660028003123E021235B4854F9975BB
:1009DE004E00754D00020B7790087DE0FEA3E0FF00
:1009EE00900073120048E599F090087D126A979076
:1009FE00087DE0FEA3E0FFAC32AD338F028E038C98
:100A0E00068D07906473126A58E493F9740193FE8D
:100A1E00EAD39EEB994009854F99754E00754D00AE
:100A2E00020B7790087DE0FEA3E0FF9000731200AA
:100A3E0048E599F090087D126A9790087DE0FEA334
:100A4E00E0FFEFB40006EEB401028003020B7790D4
:100A5E000053E0D394C7400B900053E0C394C8F505
:100A6E0050801A900053E0D39463400B900053E0F3
:100A7E00C39464F5508006900053E0F550E5507530
:100A8E00F002A4FFAEF08F73EF900073126ABAEF0C
:100A9E00FCE0FDEC900076126ABAEDFCE0FDEC2D68
:100AAE00B550028003020B680FEF900073126ABA02
:100ABE00E573FFE0FCEF900077126ABAECFFE0FC02
:100ACE00EFC39CB550028003020B68E5739000756E
:100ADE00126ABAE573FFE0FCEF900078126ABAEC86
:100AEE00FFE0FCEF2CB55072E573900079126ABAF4
:100AFE00E0C39550900899F0E57390007A126ABAA7
:100B0E00E0C3955090089AF0E57390007D126ABA92
:100B1E00E0C3955090089BF0E57390007E126ABA80
:100B2E00E0C3955090089CF0E57390007F126ABA6E
:100B3E00E0C3955090089DF0E573900080126ABA5C
:100B4E00E0C3955090089EF01201247599F97464D3
:100B5E00F5097508001200F880FE7599FF7464F5AA
:090B6E00097508001200F880FE70
:0F3280000206E102078C0209730209E6020A3115
:100B770022E54D90328FF8282873020C5C90087D8F
:100B8700E0FEA3E0FF900049120048E0F5999008C5
:100B97007D126A9790087DE0FEA3E0FF74116F4E07
:100BA7007003754D00020C5C856E99020C5C900811
:100BB7007DE0FEA3E0FF900073120048E0F599EF97
:100BC700B40107EEB40703754D0090087D126A97CC
:070BD700020C5C90087EE0B7
:0F328F00020B81020B84020BAF020BB5020BDAAC
:100BDE009032E3F82828738553998067855F998052
:100BEE0062856199805D8565998058856799805386
:100BFE00856899804E8569998049856A9980449067
:100C0E000018E0F599803CA22CB340077599FAC202
:100C1E002C8017A21FB3400575990F800B900047CB
:100C2E00E0F599900047E4F0C21F8017856B99801C
:100C3E0012856699800D856C9980087599FC8003E4
:030C4E00754D00E1
:1032E300020BE5020BEA020BEF020BF4020BF902ED
:1032F3000BFE020C03020C08020C0D020C15020C4F
:0D3303003A020C3F020C44020C49020C4E31
:0B0C510090087D126A9780031233EDBB
:03329E00020C59C6
:100C5C0022E537255BFFAE5A50010E90007312004F
:100C6C0048E0F538E537255BFFAE5A50010E0FBF53
:100C7C0000010E900073120048E0F539853F3BE50A
:100C8C0038B539058538378041E539D39538401D5D
:100C9C00E539C39538853AF0A4FFAEF0E53B8E04F8
:100CAC008F05FF126A79ED2538F537801DE538C3BD
:100CBC009539853AF0A4FFAEF0E53B8E048F05FF25
:100CCC00126A79EDF4042538F53722E539D39538D5
:100CDC00401DE539C39538853AF0A4FFAEF0E53BED
:100CEC008E048F05FF126A79ED2538F537801DE5E6
:100CFC0038C39539853AF0A4FFAEF0E53B8E048FEE
:100D0C0005FF126A79EDF4042538F5372290007945
:100D1C00E0B40170E56775F00A84FF7E008F37E55B
:100D2C006775F00A84ADF07C008D3A753F0A755AF0
:100D3C0005755B24E537C394115005120C5D8006D4
:100D4C009005A8E0F537E537900063F0E56775F09E
:100D5C000A84FF7E008F37E56775F00A84ADF07C5E
:100D6C00008D3A753F0A755A05755B5AE537C39481
:100D7C00115005120C5D80069005DEE0F537E53765
:100D8C0090000EF022900079E0B4016AE56775F0EE
:100D9C000A84FF7E008F37E56775F00A84ADF07C1E
:100DAC00008D3A753F0A755A05755B36E537C39465
:100DBC00115005120C5D80069005BAE0F5378537A9
:100DCC004BE56775F00A84FF7E008F37E56775F099
:100DDC000A84ADF07C008D3A753F0A755A05755B37
:100DEC0048E537C394115005120C5D80069005CC74
:100DFC00E0F53785374C22E55F75F00484FF7E0003
:100E0C008F37E55F75F00484ADF07C008D3A753F4B
:100E1C0004755A01755B00E537C3943F5005120CFD
:100E2C005D80069001B2E0F5378537297528009072
:100E3C000046E075F020A4FFAEF09000C4E08E04F4
:100E4C008F05FF126A798D379000ACE0D3955F5017
:100E5C0003020F099000D0E0D3955F4010ED900194
:100E6C00B3126ABAE0F52B752A00020F0690009BAC
:100E7C00E0D3955F4043E5379001B3126ABAE0F5D1
:100E8C0038E5379001D3126ABAE0F5399000D0E01A
:100E9C00F404255FF53A90009BE0FE9000D0E0F45E
:100EAC00042EF53BE538B539058538378003120C2F
:100EBC00D785372B752A008041E5379001D3126A0C
:100ECC00BAE0F538E5379001F3126ABAE0F53990DB
:100EDC00009BE0F404255FF53A9000ACE0FE900036
:100EEC009BE0F4042EF53BE538B5390585383780A1
:100EFC0003120CD785372B752A00020FB09000D344
:100F0C00E0D3955F5011E537900233126ABAE0F5E1
:100F1C002B752A00020FB090009CE0D3955F5043D4
:100F2C00E537900213126ABAE0F538E537900233D0
:100F3C00126ABAE0F53990009CE0F404255FF53AAA
:100F4C009000D3E0FE90009CE0F4042EF53BE538D5
:100F5C00B539058538378003120CD785372B752AA0
:100F6C00008041E5379001F3126ABAE0F538E537B5
:100F7C00900213126ABAE0F5399000ACE0F4042543
:100F8C005FF53A90009CE0FE9000ACE0F4042EF586
:100F9C003BE538B539058538378003120CD78537D2
:100FAC002B752A00229000E4E0F53C753F11755A30
:100FBC0002755B00AE52AF53E53C75F00FA4FDAC6F
:100FCC00F0EDD39FEC9E4021E53C8E048F05FF1283
:100FDC006A79ED75F010A4FFAEF0E55F75F0118441
:100FEC00FD7C00ED2FF53D800EE55F75F01184FF63
:100FFC007E00EF24F0F53D853D37E55F75F01184FB
:10100C00AFF07E008F3A120C5D85373EAE52AF5377
:10101C009000E4E075F00FA4FDACF0EDD39FEC9ED6
:10102C004028755A02755B10853D37120C5D853E64
:10103C0038853739AE52AF53E53C8E048F05FF121D
:10104C006AA48D3A853C3B120CD78537297528004C
:10105C00752B64752A00229000E4E0F53C753F1175
:10106C00755A02755B00AE52AF53E53C75F00FA498
:10107C00FDACF0EDD39FEC9E4021E53C8E048F053A
:10108C00FF126A79ED75F010A4FFAEF0E56175F012
:10109C001184FD7C00ED2FF53D800EE56175F0119E
:1010AC0084FF7E00EF24F0F53D853D37E56175F05A
:1010BC001184AFF07E008F3A120C5D85373EAE5234
:1010CC00AF539000E4E075F00FA4FDACF0EDD39FAE
:1010DC00EC9E4028755A02755B10853D37120C5DED
:1010EC00853E38853739AE52AF53E53C8E048F05BB
:1010FC00FF126AA48D3A853C3B120CD785372975B3
:10110C002800E56B6017E56BC394FE50109000D877
:10111C00E0B402099000C6E0D3940B50028017AEE5
:10112C0028AF29E56B126A8974E78E048F05FF12CC
:10113C006A798C288D299000AEE0B40453E55F7574
:10114C00F00484FF7E008F37E55F75F00484ADF00A
:10115C007C008D3A753F04755A01755B00E537C309
:10116C00943F5005120C5D80069001B2E0F537AE4D
:10117C0028AF29E537126A8974648E048F05FF1233
:10118C006A79AE28AF29EF2DFDEE3CFC8C288D2919
:10119C00752B64752A0022900079E0B40146E5674E
:1011AC0075F00A84FF7E008F37E56775F00A84AD11
:1011BC00F07C008D3A753F0A755A05755B00E53772
:1011CC00C394115005120C5D8006900584E0F53730
:1011DC00AE2AAF2BE5372FFF50010E7464126ACC88
:1011EC008E2A8F2B90007AE0B40146E56875F00AE0
:1011FC0084FF7E008F37E56875F00A84ADF07C00C3
:10120C008D3A753F0A755A05755B6CE537C39411B9
:10121C005005120C5D80069005F0E0F537AE2AAF54
:10122C002BE5372FFF50010E7464126ACC8E2A8F77
:10123C002B900089E0B40249E56AC3944175F0052E
:10124C0084FF7E008F37E56A75F00584ADF07C0075
:10125C008D3A753F05755A06755B00E537C39413D7
:10126C005005120C5D8006900686E0F537AE2AAF6D
:10127C002BE5372FFF50010E7464126ACC8E2A8F27
:10128C002B9000CBE0B402028003021342E55F75A1
:10129C00F01584FF7E008F37E55F75F01584ADF097
:1012AC007C008D3A753F15755A03755BF4E537C3B1
:1012BC00940B5005120C5D8006900472E0F537E536
:1012CC003775F0FFA4FFAEF09000CCE08E048F05D4
:1012DC00FF126A79ED90005CF0E56675F078A4FF7A
:1012EC00AEF074FF8E048F05FF126A798C5A8D5BF9
:1012FC0074028C068D071200398F37AC5AAD5B74B3
:10130C0004FF126AA48D3A753F04755A06755B2862
:10131C00E537C3941D5005120C5D80069006B8E0AD
:10132C00F537AE2AAF2BE5372FFF50010E74641240
:10133C006ACC8E2A8F2B900078E0B4025DE5617543
:10134C00F064A4FFAEF074081200398E5C8F5D74EB
:10135C00058E048F05FF126A798D37AE5CAF5D7414
:10136C00058E048F05FF126AA48D3A753F05755AD8
:10137C0005755BDEE537C394135005120C5D8006D2
:10138C00900664E0F537AE2AAF2BE5372FFF5001FE
:10139C000E7464126ACC8E2A8F2B9000BAE0703CCB
:1013AC00900046E075F00584FF7E008F3790004674
:1013BC00E075F00584ADF07C008D3A753F05755AEB
:1013CC0005755BC0E537C3941D5005120C5D800696
:1013DC00900650E0F537E537900064F022900081DC
:1013EC00E0B401179008A0E0252BFFAE2A50010EA7
:1013FC009000D5E0126ACC8E2A8F2B9000F9E0B4C5
:10140C0001149000FAE0A852B8000495535007E577
:10141C005FC39560400280139000A3E0252BFFAEC4
:10142C002A50010E8E2A8F2B021818900081E0B4DE
:10143C000306A228B3B3400280509008A9E07010B4
:10144C009008A3E0C39405A852B800069553400237
:10145C0080109000A3E0252BFFAE2A50010E8E2A9F
:10146C008F2B9008A9E0600D9008A3E0A852B8005B
:10147C00069553400280109000A3E0252BFFAE2A66
:10148C0050010E8E2A8F2B02181890007BE0B402AC
:10149C0002800302181890007EE0602FE567D39459
:1014AC0046402890000FE0FEA3E0FF9000B9E075E5
:1014BC00F003A4FDACF0EFD39DEE9C400E9000DD4C
:1014CC00E0A852B80005D3955350030218189000A9
:1014DC00AEE0B40302800302167C85615B755A0092
:1014EC00900085E0A852B800049553500E900086E9
:1014FC00E0A85AB80005D3955B5003021679E56154
:10150C0075F002A4FFAEF074158E048F05FF126AFD
:10151C00798C068D07900603120048FEE0FFEE90D2
:10152C00007DE0FEEF8E0088F0A4FFAEF074648EB8
:10153C00048F05FF126A798C5A8D5B900046E0751A
:10154C00F018A4FFAEF09000C4E08E048F05FF12DB
:10155C006A798C068D0790061B120048AE5AAF5B59
:10156C00E0126A8974648E048F05FF126A798C5AB2
:10157C008D5BE565A85AB80077D3955B4072E5653D
:10158C00C3955BFFE4955AFE8E5A8F5B7428BE00A0
:10159C00039F500C755B28755A00740D900047F032
:1015AC00AE5AAF5B90007EE0126A8974288E048F6D
:1015BC0005FF126A798C5A8D5BAE28AF29740A8E9E
:1015CC00048F05FF126A798D068C07AC5AAD5BCF80
:1015DC00CECF120003740A8E048F05FF126A798C29
:1015EC005A8D5BAE28AF29126AD48E288F29807D44
:1015FC00E565A85AB80004955B5072AE5AAF5BE52E
:10160C0065126ACC8E5A8F5B7428BE00039F500CF7
:10161C00755B28755A00740D900047F0AE5AAF5B9D
:10162C0090007EE0126A8974288E048F05FF126A7E
:10163C00798C5A8D5BAE28AF29740A8E048F05FF06
:10164C00126A798D068C07AC5AAD5BCFCECF1200E7
:10165C0003740A8E048F05FF126A798C5A8D5BAE67
:10166C0028AF29EF2DFDEE3CFC8C288D2902181893
:10167C009000C6E0855FF0A4FFAEF07405126A8995
:10168C0074071200398E5A8F5B900085E0A852B80F
:10169C00000495535012900086E075F002A4FDAC46
:1016AC00F0EFC39DEE9C4003021818E55F75F00B3C
:1016BC0084FF7E00900603120048FEE0FFEE9000CF
:1016CC007DE0FEEF8E0088F0A4FFAEF074648E0413
:1016DC008F05FF126A798C5A8D5B900046E075F08D
:1016EC0018A4FFAEF09000C4E08E048F05FF126AC0
:1016FC00798C068D0790061B120048AE5AAF5BE042
:10170C00126A8974648E048F05FF126A798C5A8D63
:10171C005BE565A85AB80077D3955B4072E565C365
:10172C00955BFFE4955AFE8E5A8F5B7428BE0003BE
:10173C009F500C755B28755A00740D900047F0AEE5
:10174C005AAF5B90007EE0126A8974288E048F0574
:10175C00FF126A798C5A8D5BAE28AF29740A8E04FD
:10176C008F05FF126A798D068C07AC5AAD5BCFCE14
:10177C00CF120003740A8E048F05FF126A798C5AFB
:10178C008D5BAE28AF29126AD48E288F29807DE517
:10179C0065A85AB80004955B5072AE5AAF5BE5650C
:1017AC00126ACC8E5A8F5B7428BE00039F500C7546
:1017BC005B28755A00740D900047F0AE5AAF5B90E1
:1017CC00007EE0126A8974288E048F05FF126A79F4
:1017DC008C5A8D5BAE28AF29740A8E048F05FF12CC
:1017EC006A798D068C07AC5AAD5BCFCECF12000355
:1017FC00740A8E048F05FF126A798C5A8D5BAE28A1
:10180C00AF29EF2DFDEE3CFC8C288D29229000D9C0
:10181C00E0B4026AE55F75F00884FF7E008F37E55F
:10182C005F75F00884ADF07C008D3A753F08755AF1
:10183C0001755BE0E537C3943F5005120C5D8006E3
:10184C00900272E0F53785372D752C00AE2CAF2D3C
:10185C00AC2AAD2B12000374648E048F05FF126A40
:10186C00798C2C8D2D900076E08C068D07126A8970
:10187C0074648E048F05FF126A798C2C8D2DAE2822
:10188C00AF29AC2AAD2B12000374648E048F05FFB4
:10189C00126A798C288D29900076E08C068D0712BF
:1018AC006A8974648E048F05FF126A798C288D29DD
:1018BC00A204401DAE52AF537405BE00039F5002EC
:1018CC00D204E561D394CC4008D202741190004745
:1018DC00F09000D8E0B402089000C6E0640B6002FF
:1018EC008035AE28AF29E56B126A8974E78E048FB8
:1018FC0005FF126A798C288D299000D9E0B4021763
:10190C00AE2CAF2DE56B126A8974E78E048F05FF40
:10191C00126A798C2C8D2D900098E05402601B90EB
:10192C00008FE0A852B80012D39553400DA204B317
:10193C00B35007E561C3949A40028028AE34AF35AA
:10194C0090008DE075F002A4FDACF0EF2DFDEE3CA7
:10195C00FC74022DFD50010CE561BC0007D39D40C9
:10196C0003754301856135753400E5437003021A34
:10197C005C9000EBE0C395435003021A4E9000FBC1
:10198C00E0C394025076E56775F00A84FF7E009000
:10199C000573120048E0F55B755A00AE5AAF5B90C8
:1019AC00008EE0126A8974648E048F05FF126A79C6
:1019BC008C5C8D5D9000EBE004C395438C068D0729
:1019CC00126A899000EBE08E048F05FF126A798C05
:1019DC005C8D5DAE28AF29EF2DFDEE3CFC8C288D87
:1019EC00299000D9E0B40212AE2CAF2DAA5CAB5DED
:1019FC00EF2BFBEE3AFA8A2C8B2D80469000EBE015
:101A0C0004C39543854BF0A4FFAEF09000EBE08E41
:101A1C00048F05FF126A798C5C8D5DAE28AF29EFBF
:101A2C002DFDEE3CFC8C288D299000D9E0B40212DF
:101A3C00AE2CAF2DAA5CAB5DEF2BFBEE3AFA8A2CE9
:101A4C008B2D05439000EBE0C39543500375430089
:101A5C00900098E05401601B90008CE0A852B800F4
:101A6C0012D39553400DA204B3B35007E55FC39452
:101A7C00CC4002802590008AE075F003A4FFAEF004
:101A8C00E5402FFF50010E74032FFF50010EE55F50
:101A9C00BE0007D39F4003754401855F40E5447049
:101AAC0003021B8F9000ECE0C395445003021B8192
:101ABC009000FBE0C394025076E56775F00A84FF52
:101ACC007E00900573120048E0F55B755A00AE5A23
:101ADC00AF5B90008BE0126A8974648E048F05FFF3
:101AEC00126A798C5C8D5D9000ECE004C395448C9B
:101AFC00068D07126A899000ECE08E048F05FF12A8
:101B0C006A798C5C8D5DAE28AF29EF2DFDEE3CFC27
:101B1C008C288D299000D9E0B40212AE2CAF2DAADE
:101B2C005CAB5DEF2BFBEE3AFA8A2C8B2D8046904A
:101B3C0000ECE004C39544854CF0A4FFAEF090009B
:101B4C00ECE08E048F05FF126A798C5C8D5DAE28FB
:101B5C00AF29EF2DFDEE3CFC8C288D299000D9E0AF
:101B6C00B40212AE2CAF2DAA5CAB5DEF2BFBEE3AA0
:101B7C00FA8A2C8B2D05449000ECE0C3954450035D
:101B8C007544009000EEE02529FFAE2850010E8E22
:101B9C00288F2990009DE0A828B8000495295009A9
:101BAC0090009DE0F5297528009000D9E0B4020D55
:101BBC0090009DE0A82CB80006952D40028009905D
:101BCC00009DE0F52D752C00229000D9E0B40102A7
:101BDC008003021CE0A204B35003021CDE9000A49C
:101BEC00E0B40168AE28AF29AC52AD5312000374B7
:101BFC003C8E048F05FF126A799000B4E0BC001093
:101C0C009D400D9000B6E0A828B80004952950021C
:101C1C00D203AE28AF29AC52AD53120003743C8EE4
:101C2C00048F05FF126A799000B4E0C3940ABC00DB
:101C3C0015D39D40119000B6E0C39405A828B800B8
:101C4C0005D3952950028002C2038068AE28AF29C3
:101C5C00AC52AD5312000374788E048F05FF126AD8
:101C6C00799000B4E0BC00109D400D9000B6E0A847
:101C7C0028B8000495295004D2038038AE28AF2927
:101C8C00AC52AD5312000374788E048F05FF126AA8
:101C9C00799000B4E0C3940ABC0015D39D40119018
:101CAC0000B6E0C39405A828B80005D395295002C6
:101CBC008002C203A203B34019AE28AF299000B52D
:101CCC00E0126A8974648E048F05FF126A798C287D
:101CDC008D298002C203A201B34006A202B3B35005
:101CEC0009900017E4F0A3F08024AE28AF2974000B
:101CFC00D39F74019E400C900017E528F0A3E529B2
:101D0C00F0800B74FF900017F8E4F0E8A3F090005B
:101D1C00A4E0B4011AAE28AF297402126A898E2885
:101D2C008F29AE2CAF2D7402126A898E2C8F2D90B8
:101D3C0000BBE0C39403400990006FE0C3940250D1
:101D4C0035AE28AF29745E126A89740A8E048F0529
:101D5C00FF126A798C288D299000D9E0B40217AE55
:101D6C002CAF2D745E126A89740A8E048F05FF12D3
:101D7C006A798C2C8D2DAE28AF297402BE000AD343
:101D8C009F4006752902752800AE2CAF2D7402BE3B
:101D9C00000AD39F4006752D02752C00900015E5A6
:101DAC0028F0A3E529F022900046E0900373126A14
:101DBC00BAE0F541754264900046E0FE9000AFE059
:101DCC00D39E4037E55F75F00884FF7E008F37E5C2
:101DDC005F75F00884ADF07C008D3A753F08755A3C
:101DEC0003755B96E537C3941F5005120C5D800696
:101DFC00900428E0F5378537428035E55F75F008AB
:101E0C0084FF7E008F37E55F75F00884ADF07C00B1
:101E1C008D3A753F08755A03755BB6E537C3941F49
:101E2C005005120C5D8006900448E0F5378537426A
:101E3C00229000E5E0F53C753F11755A04755B0086
:101E4C00AE52AF53E53C75F00FA4FDACF0EDD39F53
:101E5C00EC9E4021E53C8E048F05FF126A79ED75EE
:101E6C00F010A4FFAEF0E55F75F01184FD7C00ED81
:101E7C002FF53D800EE55F75F01184FF7E00EF2499
:101E8C00F0F53D853D37E55F75F01184AFF07E00D0
:101E9C008F3A120C5D85373EAE52AF539000E5E0A1
:101EAC0075F00FA4FDACF0EDD39FEC9E4028755A55
:101EBC0004755B10853D37120C5D853E38853739CE
:101ECC00AE52AF53E53C8E048F05FF126AA48D3AD7
:101EDC00853C3B120CD7853741754264229000E556
:101EEC00E0F53C753F11755A04755B00AE52AF536B
:101EFC00E53C75F00FA4FDACF0EDD39FEC9E4021BA
:101F0C00E53C8E048F05FF126A79ED75F010A4FF85
:101F1C00AEF0E56175F01184FD7C00ED2FF53D8090
:101F2C000EE56175F01184FF7E00EF24F0F53D8520
:101F3C003D37E56175F01184AFF07E008F3A120CDD
:101F4C005D85373EAE52AF539000E5E075F00FA4BF
:101F5C00FDACF0EDD39FEC9E4028755A04755B10D8
:101F6C00853D37120C5D853E38853739AE52AF53FF
:101F7C00E53C8E048F05FF126AA48D3A853C3B121A
:101F8C000CD78537417542649000E0E0B404799039
:101F9C000046E0FE9000AFE0D39E4037E55F75F061
:101FAC000884FF7E008F37E55F75F00884ADF07C08
:101FBC00008D3A753F08755A03755B96E537C394E7
:101FCC001F5005120C5D8006900428E0F53785370C
:101FDC00428035E55F75F00884FF7E008F37E55F42
:101FEC0075F00884ADF07C008D3A753F08755A0386
:101FFC00755BB6E537C3941F5005120C5D800690D7
:10200C000448E0F53785374222900079E0B4013B73
:10201C00E56775F00A84FF7E008F37E56775F00A77
:10202C0084ADF07C008D3A753F0A755A05755B12CC
:10203C00E537C394115005120C5D8006900596E0AF
:10204C00F537E5422537C39464F54290007AE0B445
:10205C00013BE56875F00A84FF7E008F37E56875F3
:10206C00F00A84ADF07C008D3A753F0A755A0575FF
:10207C005B7EE537C394115005120C5D800690060B
:10208C0002E0F537E5422537C39464F542E5412576
:10209C0042F536900081E0B4021090089FE025369E
:1020AC00FE9000D5E0F4042EF5369000D8E0D394E1
:1020BC00014040E56BC394E7501D74E7C3956BFE7C
:1020CC009008A1E08E00F5F0E884FF7E008F37E5E4
:1020DC00362537F536801CE56BC394E7FE9008A1D6
:1020EC00E08E00F5F0E884FF7E008F37E536C3956F
:1020FC0037F536A2044006E5412464F536E536D3BF
:10210C0094644009E536C39464F536800375360053
:10211C009000B1E0C3953650069000B1E0F5362240
:10212C00D201900062E0A852B800049553503E9042
:10213C000062E0A852B800049553500375360F9016
:10214C000062E004A852B80004955350037536079A
:10215C00900062E02402A852B8000495535002C2C9
:10216C0001900062E060067409900047F0C22F7E77
:10217C00017F009000B7E0126A899000C6E08E04DF
:10218C008F05FF126A79E55FBC0017D39D40139051
:10219C0000C0E0B40204D22F8002C201740A900085
:1021AC0047F0900079E0B401099000B8E0C395675E
:1021BC00400280159000CAE0A852B8000495535014
:1021CC0002C201740B900047F0900079E0B4010753
:1021DC00E567C394644002801D900110E0600D908F
:1021EC000110E0A852B80006955340028008C201C5
:1021FC00740B900047F0A20140037536009000F973
:10220C00E0B401149000FAE0A852B80004955350C1
:10221C0007E55FC39560400280209000A2E0D39454
:10222C001D400B9000A2E0C3941EF536800375365A
:10223C00007415900047F002231D900081E0B40358
:10224C0006A228B3B3400302231D9008A3E0C39455
:10225C0005A852B80004955350069008A9E06002F6
:10226C00801D9000A2E0D3941D400B9000A2E0C30F
:10227C00941EF5368003753600740C900047F09070
:10228C0008A3E0A852B80004955350069008A9E0A2
:10229C007002801D9000A2E0D3941D400B9000A210
:1022AC00E0C3941EF5368003753600740C9000471D
:1022BC00F09008A3E0A852B8000495535031900058
:1022CC00C0E0B40228D22F9008A8E0FE9008A9E044
:1022DC00D39E50069008A9E0700280099008A8E4EB
:1022EC00F0C22F80069008A8E004F08002C2019092
:1022FC0008A3E02405A852B800049553501390008D
:10230C00C0E0B4020A9008A9E07002D22F8002C289
:10231C0001A22EB3401D9000A2E0D3941D400B905F
:10232C0000A2E0C3941EF53680037536007410903D
:10233C000047F085366C9000A2E0D3941D401890B5
:10234C000070E02536FE900046E075F01E84FC7FA0
:10235C0000EE2CF5368049900047E0640C600F903D
:10236C000047E064106007900047E0B41516900039
:10237C0070E0FE900046E075F01E84FC7F00EE2CB1
:10238C00F536801C900072E02536FE900070E02E31
:10239C00FE900046E075F01E84FC7F00EE2CF536B6
:1023AC0022900046E075F00584FF7E008F37900088
:1023BC0046E075F00584ADF07C008D3A753F0575EF
:1023CC005A03755BD69000C4E01475F00584FF7E4B
:1023DC0000E537BE00039F5005120C5D800BE537FE
:1023EC00900449126ABAE0F537E5379008A2F090EC
:1023FC0008A2E0FE9000B3E0C39E50089000B3E04A
:10240C009008A2F022E56775F00A84FF7E00900523
:10241C0073120048E0F546E546D394644010E54657
:10242C00C3946475F00F84FF7E008F46800375465D
:10243C0000900096E02546F54622E56775F00A8483
:10244C00FF7E00900573120048E0C39469505590CC
:10245C0000E0E0C394035026900875E0FEA3E0FF73
:10246C007404120039E55F126A89740F8E048F05AB
:10247C00FF126A79900873ECF0A3EDF080249008B9
:10248C0075E0FEA3E0FF7404120039E561126A895D
:10249C00740F8E048F05FF126A79900873ECF0A309
:1024AC00EDF0800F900875E0F8A3E0900873C8F089
:1024BC00A3C8F0A204401A900875E0FEA3E0FF74D4
:1024CC0003126A897401120039900873EEF0A3EFBD
:1024DC00F0900873E0FEA3E0FF900879E0FCA3E025
:1024EC00FDEDD39FEC9E400F900879E0F8A3E090AF
:1024FC000873C8F0A3C8F0900089E0B40262E56AE2
:10250C00C3944175F00584FF7E008F37E56A75F042
:10251C000584ADF07C008D3A753F05755A06755BE8
:10252C0014E537C394175005120C5D800690069A7B
:10253C00E0F537900873E0FEA3E0FF740A8E048F79
:10254C0005FF126A79E5378C068D07126A89740AC1
:10255C008E048F05FF126A79900873ECF0A3EDF0EE
:10256C0022E50875F004A4FFAEF09006B612004800
:10257C00E09032A1F8282873804C855373804790E3
:10258C0000C6E0855FF0A4FFAEF074081200398F2E
:10259C00738033856173802E85677380298568739A
:1025AC008024856973801F856A73801A856B73809C
:1025BC00158566738010856573800B856C7380063A
:0625CC00900018E0F57319
:1032A10002258402258602258B02259F0225A40280
:1032B10025A90225AE0225B30225B80225BD0225A6
:0732C100C20225C70225CC63
:1025D200E50875F004A4FFAEF09006B7120048E5D6
:1025E2000875F004A4FFAEF0E0FC9006B8120048B3
:1025F200ECFEE0FFEEC39F40030226DAE50875F029
:1026020004A4FFAEF09006B6120048E0B40441E51F
:102612000875F004A4FFAEF09006B8120048E0C3BB
:102622009573500AE508F50CD39230124134E5084F
:1026320075F004A4FFAEF09006B7120048E0D395FF
:1026420073400AE508F50CC392301241340226D8D1
:10265200E50875F004A4FFAEF09006B7120048E05A
:10266200C395735015E50875F004A4FFAEF090060B
:10267200B8120048E0D395735002800AE508F50CC1
:10268200D39230124134E50875F004A4FFAEF09005
:1026920006B7120048E0D395735015E50875F004AB
:1026A200A4FFAEF09006B8120048E0C39573500A3A
:1026B200E508F50CC392301241349006BEE0B40135
:1026C200099000D2E0D395615002800A7402F50CA1
:1026D200C39230124134806AE50875F004A4FFAE5B
:1026E200F09006B7120048E0D395734015E50875DF
:1026F200F004A4FFAEF09006B8120048E0C3957350
:102702004002800AE508F50CC39230124134E50814
:1027120075F004A4FFAEF09006B7120048E0C3952E
:10272200734015E50875F004A4FFAEF09006B812E8
:102732000048E0D39573400AE508F50CD3923012B5
:10274200413422AE2EAF2F74C9BE000CD39F400875
:10275200782E126ADC02285F752F01752E00AE52A8
:10276200AF53E546BE000DD39F40099000A8E0D3C9
:10277200954740028023754700E546C39553F5739C
:102782009000ABE0D395454008E5452573F54580BB
:10279200069000ABE0F54580020547900084E0D347
:1027A2009561401CE55FC395604015AE52AF53E59D
:1027B20046BE00039F50099000A9E0D3954840020D
:1027C200806E9008A4E0A852B80004955350037597
:1027D2004A009008A4E0A852B8000BD395534006D3
:1027E200E5539008A4F0E54A7041E553C39546F5D8
:1027F20073E573D3940540037573059000AAE0C393
:1028020095455007E573C3954540028009E545C3E8
:102812009573F54580069000AAE0F5459000AAE080
:10282200D3954540069000AAE0F545754800800220
:102832000548E54A7016900084E0C39561500DE5A5
:10284200462405A852B8000695534002800F900016
:1028520097E0F545754A0174789008A4F022AE2EEF
:10286200AF2F74E9D39F74039E4008782E126ADC5E
:10287200022A06752F01752E00754532A229402ABB
:10288200754519900097E075F002A4FFAEF0E54798
:10289200BE0006D39F4002D2290547754A037478C9
:1028A2009008A4F07549000229EDAE52AF53E546F7
:1028B2006F4E70030229EDE546BE000DD39F40091D
:1028C2009000A8E0D395474002800F754700E54A83
:1028D200C394035003754519800DE546C39553F51E
:1028E20073E5472573F547900084E0D39561400E68
:1028F2009008A4E0A852B80007D395534002800C78
:102902000549900097E0B54903754A00E54AB403CA
:1029120006A204B3B34002800A0549E549B43C0368
:10292200754A02E54AB402299008A4E0A852B80008
:102932000ED395534009E5539008A4F075490090D1
:102942000084E0C39561500975490074789008A429
:10295200F0E54A705A900084E0D39561401CE55F2F
:10296200C395604015AE52AF53E546BE00039F507B
:10297200099000A9E0D39548400280087548007587
:10298200454B8028E553C39546F573E573D394050B
:102992004003757305900084E0D395614008E548D3
:1029A2002573F5488006E5482406F548754900E593
:1029B2004A7016900084E0C39561500DE5462405E7
:1029C200A852B80006955340028003754A01E54AB1
:1029D200B401187545190549900097E0B549067587
:1029E2004A0275490074789008A4F0A202B3400329
:1029F200754532E54575F00AA4FFAEF090087BEE0E
:102A0200F0A3EFF022E56F9032C8F8282873900007
:102A12007CE07003022C449000B2E0B40102800317
:102A2200022B4F900044E0655E6009E55345526019
:102A320003022B4C7E017F00E5BE126A89E5BD2FA1
:102A4200FF50010E8E5A8F5B7410126A89900061DA
:102A5200E08E048F05FF126A7990087FECF0A3EDF7
:102A6200F0E56B600FE56BC394FE50089000D8E070
:102A72006402600280649000C6E0B40B1F90087F7D
:102A8200E0FEA3E0FF74E7126A89E56B8E048F050E
:102A9200FF126A7990087FECF0A3EDF09000C6E097
:102AA200D3940B40089000AEE064046002802B9047
:102AB200087FE0FEA3E0FF900883E0FCA3E0FDEFC7
:102AC200D39DEE9C400D126AD490087FEEF0A3EFE6
:102AD200F0800790087FE4F0A3F090007CE0B4025D
:102AE20027900881E0FEA3E0FF90087FE0FCA3E0CE
:102AF200FDEF2DFDEE3CFC74018C068D07120039B2
:102B020090087FEEF0A3EFF090087FE0FEA3E0FFD5
:102B1200900881E0FCA3E0FDEDD39FEC9E4004D23F
:102B22002D8002B22D90087FE0F8A3E0900881C8C2
:102B3200F0A3C8F09000AEE064016006A22DB3B32A
:102B420040028006900880E0F55F022C42D22D7E82
:102B5200017F00E5BE126A89E5BD2FFF50010E8E8E
:102B62005A8F5B7410126A89900061E08E048F059F
:102B7200FF126A7990087FECF0A3EDF0E56B600F2D
:102B8200E56BC394FE50089000D8E06402600280B6
:102B9200649000C6E0B40B1F90087FE0FEA3E0FF44
:102BA20074E7126A89E56B8E048F05FF126A7990C9
:102BB200087FECF0A3EDF09000C6E0D3940B400840
:102BC2009000AEE064046002802B90087FE0FEA3D8
:102BD200E0FF900883E0FCA3E0FDEFD39DEE9C4074
:102BE2000D126AD490087FEEF0A3EFF080079008F0
:102BF2007FE4F0A3F090007CE0B40227900881E02B
:102C0200FEA3E0FF90087FE0FCA3E0FDEF2DFDEEC8
:102C12003CFC74018C068D0712003990087FEEF09F
:102C2200A3EFF090087FE0F8A3E0900881C8F0A33A
:102C3200C8F09000AEE064016006900880E0F55FA5
:102C42008003755F00900078E07006756F01022ABC
:102C52000775BB1802327B900078E07003022DCA20
:102C62007E017F00E5BE126A89E5BD2FFF50010E8D
:102C72008E5A8F5B9000BEE0B4010F7E0F7FFFACD7
:102C82005AAD5B126AD48E5A8F5B9000E3E0B402B5
:102C920045AE5AAF5B900021E0FCA3E0FDEDD39F6F
:102CA200EC9E400A900021E55AF0A3E55BF0AE5A93
:102CB200AF5B900023E0FCA3E0FDEFD39DEE9C40D0
:102CC2000A900023E55AF0A3E55BF0AE5AAF5B74BD
:102CD200041200398F619000E3E0704CAE5AAF5B92
:102CE200900021E0FCA3E0FDEFD39DEE9C40091291
:102CF2006AD48E5A8F5B8006755B00755A00AE5A95
:102D0200AF5B7410126A8990005EE08E048F05FF3B
:102D1200126A798C5A8D5B74FFBC0009D39D400501
:102D2200855B6180037561FE9000AEE0B4010280B4
:102D320003022DC8A204B3B3500E900082E0A85241
:102D4200B80005D39553500280719000BFE08561B1
:102D5200F0A4FFAEF074648E048F05FF126A798CC2
:102D62005A8D5BE56B6016E56BC394FE500F9000C5
:102D7200D8E0B402089000C6E0640B60028017AE8F
:102D82005AAF5B74E7126A89E56B8E048F05FF12F6
:102D92006A798C5A8D5BAE5AAF5B90087FE0FCA3D8
:102DA200E0FDEDD39FEC9E4005855B5F800BA22D7D
:102DB200B34006900880E0F55F800BA22DB3400679
:102DC200900880E0F55F800375610090007BE07001
:102DD20006756F02022A0775BB1902327B90007BCF
:102DE200E07003022E7FE55ED395514003022E7DF3
:102DF20090001FE0FEA3E0FFE565126ACC90001F81
:102E0200EEF0A3EFF07E017F00E5BE126A89E5BD18
:102E12002FFF50010E8E5A8F5B9000E8E070137402
:102E22000A126A8974518E048F05FF126A798D65C0
:102E32008019AE5AAF5B740A126A898F048E057EBE
:102E4200017F95CDCCCD1269778F65E565D394640A
:102E5200400375656490001FE0FEA3E0FFE5652F67
:102E6200FF50010E90001FEEF0A3EFF090007FE004
:102E7200048E048F05FF126A798D658003756532B1
:102E82009000CBE07006756F03022A0775BB130230
:102E9200327B9000CBE0604A7E017F00E5BE126A81
:102EA20089E5BD2FFF50010E8E5A8F5B740412000C
:102EB200398F669000CDE08566F0A4FDACF07464B5
:102EC200FF126A798D669000CCE08566F0A4FFAEB1
:102ED200F074FF8E048F05FF126A79ED90005DF0A9
:102EE2008003756600900079E07006756F04022A0F
:102EF2000775BB1702327B900079E0B401028003B0
:102F0200022F8D7E017F00E5BE126A89E5BD2FFF8B
:102F120050010E8E5A8F5B9008A5E060199008A5AB
:102F2200E0149064B712008CE493FC740193FDEDFD
:102F3200C39FEC9E400280069008A5E014F0900822
:102F4200A5E0C394B3501DAE5AAF5B9008A5E00450
:102F52009064B712008CE493FC740193FDEFC39D5F
:102F6200EE9C400280069008A5E004F09008A5E0DF
:102F7200FE90009FE08E0088F0A4FFAEF074648E95
:102F8200048F05FF126A798D6780037567009000D0
:102F92007AE07006756F05022A0775BB1602327B4E
:102FA20090007AE0B4010280030230367E017F0095
:102FB200E5BE126A89E5BD2FFF50010E8E5A8F5B66
:102FC2009008A6E060199008A6E01490662112000D
:102FD2008CE493FC740193FDEDC39FEC9E40028050
:102FE200069008A6E014F09008A6E0C394B3501D22
:102FF200AE5AAF5B9008A6E00490662112008CE402
:1030020093FC740193FDEFC39DEE9C4002800690F9
:1030120008A6E004F09008A6E0FE9000A5E08E006D
:1030220088F0A4FFAEF074648E048F05FF126A79F3
:103032008D68800375680075BB1F02327B7E017F3D
:1030420000E5BE126A89E5BD2FFF50010E8E5A8F30
:103052005B7409126A8974E68E048F05FF126A791D
:103062008D6A900081E07006756F07022A0775BBB2
:103072001502327B900081E070030231C77E017F2E
:1030820000E5BE126A89E5BD2FFF50010E8E5A8FF0
:103092005B74041200398F69900081E0B4011590CD
:1030A20000D5E08569F0A4FFAEF07407120039EF95
:1030B2009008A0F0900081E0B402159000D5E08560
:1030C20069F0A4FFAEF07407120039EF90089FF088
:1030D200900081E0B4030280030231AA9000C2E0B2
:1030E2007052E569C39419500FD2289000A1E09064
:1030F20008A3F09008A7E4F0E569D394644004A221
:10310200284002802D9008A7E004F09008A7E0FE76
:10311200900114E0B5060B9008A3E004F09008A714
:10312200E4F09008A3E064966006900114E0700257
:10313200C22880639000A1E070349000D5E08569D8
:10314200F0A4FFAEF074FF8E048F05FF126A79EDD2
:103152009008A3F0AE52AF53741EBE0006D39F4038
:1031620002D228E561D394E54002C2288029E569AC
:10317200C3940A500DAE52AF53741EBE0004D39FC7
:1031820050028002D228E561D394E54002C2289021
:1031920000A1E09008A3F09008A3E0C394055006B4
:1031A20074059008A3F0C22E900081E0B40414E5E7
:1031B20069C394195002D22EE569D394324002C2F7
:1031C2002EC22880037569009000D8E07006756FE2
:1031D20008022A0775BB1402327B9000D8E0700304
:1031E20002326A7E017F00E5BE126A89E5BD2FFFC9
:1031F20050010E8E5A8F5B9000FDE07025EFD39444
:1032020021EE940E4005756BFF8015AE5AAF5B74CC
:1032120010126A8974E38E048F05FF126A798D6B2E
:103222008027AE5AAF5BEFD39449EE940640057502
:103232006BFF8015AE5AAF5B7410126A8974658E8B
:10324200048F05FF126A798D6BE56B75F00BA4FF95
:10325200AEF09000C6E08E048F05FF126A799008E6
:1032620083ECF0A3EDF08003756B0090007CE060CE
:093272000575BB1A800375BB1839
:1032C800022A10022C59022DDF022E94022EF90236
:0B32D8002FA202303F0230760231DCF2
:05327B00056FD2EC22FA
:096ABA002582F5825002058322B9
:0F008C0025E050020583258250020583F582226C
:106A5800EF2F500205832582F582E5833E2EF583CC
:016A6800220B
:106ACC00CFC39FFF50011E22C3EF9DFFEE9CFE2201
:086ADC000806B60002180622AC
:0D6A9700A3E004F07006126AB0E004F022E3
:0E003900048007C3CE13CECF13CFD5E0F6223E
:10697700BC000FBE0008ED8FF084FFADF022E4FEEF
:10698700FF22BE000DEF60FE54F0606F20E70302A8
:106997006A2DEAC0E0EBC0E078017A0075F001EEFD
:1069A70020E710EF25E0FFEE33FE0AC5F023C5F020
:1069B70030E7F0EA5407F9096A7A007B00600108BA
:1069C700C3EC9E40167004ED9F4010ED9FFDEC9EBA
:1069D700FCE5F0CA4ACA03F5F08005E5F003F5F0D7
:1069E700C3EE13FEEF13FFD9D77908CACBCAD8D0A5
:1069F700EAFEEBFFD0E0FBD0E0FA22EC8FF084FC5C
:106A0700ED54F045F0C48FF084FEEDC454F045F02A
:106A1700C48FF084FDEEC4FE54F02DFFEE540F3CFE
:106A2700FEADF07C0022790078008FF0EC7E082024
:106A3700E70DC3CD33CD33C933C9C833C8DEF084BE
:106A470049F9E5F08FF0BE00E6FD7C00E9FFE8FEBE
:016A5700221C
:0E6A8900F88FF0A4FFE5F0CE88F0A42EFE22D8
:10000300EF8DF0A4F9A8F0EF8CF0A428F8EE8DF0B2
:06001300A428FEE9FF2213
:106A6900600D782B026A73007830D8FED5E0F822E1
:106A7900EEC0E07E00126977EFFDEEFCD0E0FE2269
:0C6AA400EEC0E07E00126977D0E0FE2218
:03001B0002001EC2
:0300530002005652
:03009B00020071EF
:03000000026AC3CE
:096AC30075817575D0000243D005
:0B004800E5822FF582E5833EF5832260
:0A6AB0000582D582021583158222AB
:10001E00C0E0C0F0C083C082C0D075D0001242CE06
:0B002E00D0D0D082D083D0F0D0E032E0
:10005600C0E0C0F0C083C082C0D075D0001242D1CB
:10006600D0D0D082D083D0F0D0E032C0E0C0F0C093
:1000760083C082C0D075D000124392D0D0D082D037
:0600860083D0F0D0E0324F
:00000001FF
